:102000000030002051B800004590000045900000CD
:1020100000000000000000000000000000000000C0
:1020200000000000000000000000000045900000DB
:102030000000000000000000459000007124000036
:10204000459000004590000045900000459000003C
:10205000459000004590000045900000459000002C
:10206000459000004590000045900000459000001C
:10207000E124000045900000459000000D2A00007A
:1020800045900000459000004590000045900000FC
:1020900045900000459000004590000045900000EC
:1020A00045900000459000004590000045900000DC
:1020B00045900000459000004590000045900000CC
:1024100010B5064C2378002B07D1054B002B02D0BA
:10242000044800E000BF0123237010BD94F0FF1F9B
:102430000000000038C00000084B10B5002B03D08E
:102440000749084800E000BF07480368002B00D197
:1024500010BD064B002BFBD09847F9E700000000A9
:1024600098F0FF1F38C0000090F0FF1F0000000030
:102470000E4A1368013313600D4A13680133136069
:102480000C4B1A68002A08D01A68013A1A601B68B7
:10249000002B02D10122084B1A70084B1A68002A3F
:1024A00002D01A68013A1A607047C046B0F0FF1FA8
:1024B00044F5FF1FD4F4FF1FD0F4FF1FD8F4FF1F13
:1024C000FA22034B92015A6007221A607047C046F5
:1024D00010E000E0014B18687047C046B0F0FF1FE5
:1024E00030B5244B1A79D2B2910614D52249086826
:1024F0000130202800D100204C68A04205D00C6893
:10250000DD790C19EDB22572086005241B480460C2
:10251000886A1B4908604020024206D0802419497D
:1025200064058C60D9788143D97052B2002A1CDAD4
:10253000134A1068002818D10F4AD46A116B8C42D4
:1025400014D080240F4964054C60116B4C1C14633B
:1025500014003434615CC9B2D971116B202900D1E7
:1025600010634022D9780A43DA7030BD7F21DA78CF
:102570000A40F9E700A00640B4F0FF1FD4F4FF1FA3
:10258000D8F4FF1F00F00F4080221E4B5203596900
:1025900010B50A435A618022D9681B4C0A43DA609D
:1025A0005A681A490A405A605A6819490A405A60DA
:1025B0005A6818490A405A600023E370A370A37157
:1025C00063710B2800D91800134B8000C158962363
:1025D0001B02994214D9114B4808C01806F01EFE80
:1025E0001F21227880B2030A0B408A4313432370D1
:1025F0002C23C0B26070E3700C2006F033FD10BDD8
:102600000648EBE70080044000A00640FFFCFFFF07
:10261000FFEFFFFFFF7FFFFF64BE000040420F009F
:102620000A4A10B5D36A0133202B00D10023116B65
:102630008B4209D01400D16A343460548021D362B3
:10264000034AD3780B43D37010BDC046B4F0FF1FCC
:1026500000A006400A4B10B55C68196800228C4245
:102660000BD05A68511C59609A18127A5968027036
:102670000122202901D100215960100010BDC0465F
:10268000B4F0FF1F014B98627047C046B4F0FF1FC3
:102690000020034B1A78824201D018700130704735
:1026A000D0F4FF1FBFF34F8F024A034BDA60BFF332
:1026B0004F8FFEE70400FA0500ED00E02E4B2F4A95
:1026C000F0B55A612E4A80205A602E4A2E499A60EF
:1026D00000229A614861486080208A612B4980030A
:1026E0004A618A612A49082488600720C86029490C
:1026F0000A2548681600A043140085B0264F48609C
:1027000001911020986003960398B84229D980213E
:10271000186949030840414241418C4610216444F4
:10272000596003960398B8421FD98021186949035C
:102730000840411E8841013D1218002DE1D1174883
:102740000A2C16D10A2A14D1093A0270019A019969
:102750005068082202434A608022D2005A6005B0C5
:10276000F0BD039801300390CEE703980130039049
:10277000D8E70022E9E7C04600F00F40132C051807
:10278000002805080304001040F00F4080F00F40BF
:102790000090044000800440E703000080F9FF1F20
:1027A000002802D0012804D070470122024B9A6011
:1027B000FAE70222FAE7C04600F00F40002802D0F4
:1027C000012804D070470122024B5A60FAE7022226
:1027D000FAE7C04600F00F4000B50A281DD806F001
:1027E00009FD060D10141C1C1C1C1C1C18000C4B95
:1027F0001B880C4898428041404200BD084B5B88D2
:10280000F7E7094B1869C00FF7E7074B1869400055
:10281000F9E7054B18698000F5E70020EDE7C046B1
:1028200008F1FF1FFF03000000F00F40002803D055
:10283000012806D0002003E0044B1868012318404B
:102840007047024B1B685B08F9E7C04600F00F4079
:1028500070B50500002401263300A340E0B21D42FC
:1028600005D0FFF7ABFF0134202CF5D170BDFFF789
:1028700097FFF8E770B5002401262500E0B2FFF7C6
:10288000ABFF002802D03300A3401D430134202CAD
:10289000F4D1280070BD704780230D4A9B05516913
:1028A00010B50B4353613C220A4B0F209A61333A17
:1028B0009A6000225A600332DA601A60013A1A60A4
:1028C00002321A6041321A6006F0CCFB10BDC046DD
:1028D0000080044000B00340F8B5092859D806F03C
:1028E00089FC05085858585858580B132A4B188813
:1028F000F8BD294B5888FBE7274B28489B88284977
:10290000584306F015FDF3E7234BD88807F00EF87F
:1029100008F0C2FD0022234B07F092FF0022224B59
:1029200007F08EFF04000D0002000B0000201E497E
:1029300008F006FA1D4A06000F001D4B2000290072
:1029400007F04AFB02000B003000390007F044FB9F
:1029500008F0F4FD08F0A0FD0022164B07F03CFB48
:1029600008F0E8FF144A154B07F06AFF0022144BE9
:1029700007F022F802000B001248134907F02CFB65
:102980000D4A124B08F0DCF908F0D8FD06F0FAFD0C
:10299000AEE70020ACE7C04608F1FF1F850200004B
:1029A000FF0F00000000303F00001440CDCCCCCC25
:1029B000CCCC124000002440C3F5285C8FA27240AA
:1029C00000FEAA409A999999FD6F2F418F1271408C
:1029D0000C4B82B01B78002B11D000220A490192C7
:1029E000019B8B4207D90192019B8B42F7D8019B37
:1029F00001330193F8E7019B01330193F0E702B043
:102A00007047C04680F9FF1F3F0D0300094B0A4A7B
:102A10001969118019695180196991801969D180EA
:102A200003221A60013A1A6002321A6041321A60B7
:102A30007047C04600B0034008F1FF1F37B5802241
:102A400004000D00114BD202002915D09A6000211C
:102A5000012205F0DFFD442262430D4B9B189A7A58
:102A6000D20801925B7ADB08009300231A00102140
:102A7000200005F08BFD37BD5A60064A05F0CAFDFF
:102A80001F232A00019300932B00F0E700F00F4072
:102A900084F9FF1F0100010004220B4B186910404C
:102AA000411E88411969C000890700D510431B6980
:102AB000DB0701D502231843044B1B699B0201D598
:102AC000012318437047C04640F00F4000F00F400C
:102AD000002330B501251A000D490E480B704B70CC
:102AE0006D4204319C00C254013365502F2BF9D143
:102AF000094B19005A649A644C331A70074B4031E1
:102B00001A60074B0A701A60064B1A6030BDC04647
:102B100010F1FF1F42FAFF1F90F1FF1F3CF5FF1F4E
:102B200050F5FF1FE4F4FF1FF8B5874CA07800288C
:102B300000D004E16378012B50D0002B03D0022B8E
:102B400000D1B5E0F8BD814A18001370804A012118
:102B500013708022120504F0A3FF4422A0787D4B5D
:102B600042439B18DB7D0522002B00D0062220214A
:102B700004F034FFA078784D2B5C002B09D0774B04
:102B800082009B181A6D242104F028FF0022A378EC
:102B9000EA548022A0785205072104F08EFF4C23CE
:102BA000A0786F4A434325799E5CE2782D026179D3
:102BB000A3791543002E08D10A042A431B061A43A1
:102BC000372104F00BFFA0785CE009041A06654B7E
:102BD0000D4381002A43CD585219F1E75B4A190091
:102BE00010705B4A10708022120504F059FF4422D5
:102BF000A078584B42439B18DB7D0522002B00D068
:102C00000622202104F0EAFE544FA0783B00543302
:102C10001B5C012B3CD0002B03D0022B3AD00026AA
:102C200003E0372104F0FEFE06008022A078520562
:102C3000072104F042FFA078474D2B5C002B08D001
:102C40008300FF183A6D242104F0C8FE0022A37807
:102C5000EA542079E57800022843657937212D046C
:102C60002843A5792D060543AD19A0782A0004F064
:102C7000B5FE4C23A0783A4A43439A5C3A4B002A6B
:102C800011D15D6080220121120504F016FF59E781
:102C90002121C7E7502104F0C5FEA378334A9B00E9
:102CA0009E58861BC1E72F4A81008A58AD1AE8E773
:102CB0008022264B12051870254B0121187004F054
:102CC000FCFE4422A078234B42439B18DB7D052267
:102CD000002B00D00622202104F080FEA0781E4D9B
:102CE0002B5C002B09D01D4B82009B181A6D2421F0
:102CF00004F074FE0022A378EA548022A0785205E2
:102D0000072104F0DAFE4C23A078154A43432579C5
:102D10009F5CE6786279A3792D023543120415434E
:102D20001B062B43C31812499B00002F01D1CA5820
:102D300046E7CA580B4B8500EB58D21840E70422EF
:102D4000094B1A70FEE6C046DCF4FF1F81F9FF1F35
:102D500071F9FF1F84F9FF1F72F9FF1F90F1FF1F28
:102D6000C8F9FF1F60F9FF1F48F5FF1F74F9FF1F27
:102D7000E8F4FF1F70B5044D044CAB78002B01D074
:102D800000F02AFC04E0C046DCF4FF1F48F5FF1FFA
:102D90006360687806F038FAED0103021602320229
:102DA0003C02420246024A024E0256025D0265029F
:102DB0006D027F029102A802B102B502B902C202FD
:102DC000C602CF02D302D902DF02E502EB02F10212
:102DD000F70209031D041D041D0411031B031D0438
:102DE0001D041D041D041D041D041D041D041D04DB
:102DF0001D041D041D041D041D041D041D041D04CB
:102E00001D041D041D041D041D041D041D041D04BA
:102E10001D041D041D041D041D041D041D041D04AA
:102E20001D041D041D041D041D041D041D041D049A
:102E30001D041D041D041D041D041D041D041D048A
:102E40001D041D041D041D041D041D041D041D047A
:102E50001D041D041D041D041D041D041D041D046A
:102E60001D041D041D041D041D041D041D041D045A
:102E7000230327032B032F03330337033B033F03B2
:102E8000430347034B034F03530357031D045B03E3
:102E90006103650369036D031D0472031D041D04B2
:102EA0001D0476037B031D047F03840389031D0433
:102EB0001D048D0395039D03A5031D041D041D041E
:102EC0001D041D041D041D041D041D041D041D04FA
:102ED0001D041D041D041D041D041D040001140116
:102EE00019011E012D013C01410146014B01500118
:102EF00055015A015F011D041D041D041D046401D8
:102F00006901710178011D04930198019D01B801C7
:102F1000BD01C201C801D901DE01AD03B103B8038F
:102F2000BF03C3031D041D04C703CB03D003E30188
:102F3000E8011D04D403D803EB03EF03FA031D04D7
:102F4000FE031D0402041D041D041D041D041D04B4
:102F50001D041D041D041D041D041D041D041D0469
:102F60001D041D041D041D041D041D041D041D0459
:102F70001D041D041D041D041D041D041D041D0449
:102F80001D041D041D041D041D041D041D04060450
:102F90001D040E0414041904002005F0E1FC606017
:102FA000C84B1B78002B0AD0C74B616808221960F8
:102FB000C64B002900D012E319680A431A6070BD9D
:102FC000002005F0F7FC6060EAE7002005F000FD56
:102FD0006060E5E7002005F0EDFC002804D1A8784A
:102FE00005F010FD6060DBE7A87805F0F8FC606094
:102FF000D6E7002005F0DEFC002804D1A87805F013
:10300000A8FC6060CCE7A87805F0F5FC6060C7E735
:10301000002005F097FC6060C2E7002005F0AEFDDF
:103020006060BDE7002005F086FD6060B8E7002025
:1030300005F088FD6060B3E7002005F075FD606075
:10304000AEE7002005F085FD6060A9E7002005F0EF
:103050009CFD6060A4E7002005F082FD60609FE7B2
:10306000002005F0D3FC60609AE76F21002005F096
:10307000FFFAC002C00E606092E7954B954A9B6DC7
:103080001069984760608BE71421002005F0F0FA82
:10309000011E11D0904806F0C1F860604423AA7860
:1030A0005A438C4B9B181B7E002B00D078E760683E
:1030B00004F056FE606073E7884B6360EEE7002023
:1030C00005F07FFC60606BE7002005F050FC60605D
:1030D00066E71321002005F0CBFA011E11D07E48CF
:1030E00006F09CF860604423AA785A43794B9B18F9
:1030F0001B7E002B00D053E7606804F031FE606057
:103100004EE7764B6360EEE7002005F0D6FD606089
:1031100046E7002005F0D8FD606041E771210020FE
:1031200005F0A6FA60603BE70021080005F0A0FA70
:10313000430700D448E1A8786F2105F099FA4304C9
:1031400000D441E1012363602AE7002005F0AEFDD1
:10315000606025E7002005F0A2FD606020E7002008
:1031600005F096FD60601BE7002005F08AFD6060B9
:1031700016E7002004F084F8002805D1A87837214C
:1031800004F050FC60600BE7A878372104F04AFC9B
:10319000AB78534A9B009B58C01A606000E7514BC4
:1031A00021211878002803D104F03CFC6060F7E688
:1031B000002004F037FCAB78494A9B009B58C01AAA
:1031C0006060EDE62221002004F02CFC404B00283A
:1031D00009DBA878242182009B189D6D04F022FC55
:1031E000A8476060DCE6A878242182009B189D6DCA
:1031F00004F018FCA84740426060D1E6344B22211D
:1032000000209D6D04F00EFC0002A8476060C7E638
:103210002F4B9A6D186D90476060C1E62D4BDB6AAD
:103220006360BDE62B4B5B7A6360B9E6294B9B7A02
:103230006360B5E60F21002004F0F4FB0123184081
:103240006060ADE6002004F077FD431E98416060A9
:10325000A6E60F21002004F0E5FBC005C00F60606A
:103260009EE60F21002004F0DDFB0006C00F606029
:1032700096E60121002004F0D5FB830703D5012346
:10328000626813436360030700D489E6022362681F
:103290001343636084E60121002004F0C3FB012393
:1032A000184202D0626813436360430700D477E694
:1032B000022362681343636072E6064BDB7D636042
:1032C0006EE6C04640F5FF1F3CF5FF1FE4F4FF1F0C
:1032D00090F1FF1F84F9FF1F0024F400FFFFFF009F
:1032E00060F9FF1FC8F9FF1FBF4B252100209D6D0E
:1032F00004F098FBA847606052E6BC4B5B6B6360D0
:103300004EE6BA4B1B6B63604AE6B74B27210020A1
:103310009D6D04F087FBA847606041E6B34B9B6B53
:1033200063603DE6B04B262100209D6D04F07AFBE2
:10333000A847606034E6AD4BDB6B636030E62D215F
:10334000002004F06FFB60602AE62E21002004F0CC
:1033500069FB606024E62F21002004F063FB6060BD
:103360001EE63021002004F05DFB606018E633218A
:10337000002004F057FB606012E63421002004F0C6
:1033800051FB60600CE60121002004F04BFB43067A
:1033900003D50123626813436360030600D4FFE58D
:1033A0000223626813436360FAE50121002004F000
:1033B00039FB8005800F6060F2E50121002004F0F8
:1033C00031FBC30600D5BDE600236360E8E50121BB
:1033D000002004F027FB830600D5B3E6F4E7844B16
:1033E0005B686360DCE5824B9B686360D8E5804B7B
:1033F0001B7B6360D4E57E4BDB896360D0E57C4B4F
:103400001B696360CCE57A4B1B7D6360C8E5784B34
:103410005B7D6360C4E5764B1B6A6360C0E5744BFB
:103420005B6A6360BCE5724B9B6A6360B8E5704B96
:10343000DB6A6360B4E56E4B1B6B6360B0E56C4B9D
:103440009B696360ACE56A4BDB696360A8E57C213E
:10345000002004F0E7FA6060A2E5654B5B6B6360F7
:103460009EE5634B9B6B63609AE5614B9B7D63605C
:1034700096E55D4B54331B78636091E55C4B1B789C
:1034800063608DE5002003F0FBFE606088E5584B2B
:10349000DB6B636084E5564B40331B7863607FE5EC
:1034A000534B41331B7863607AE5514B5B6C63602F
:1034B00076E50321002004F0B5FA07231840606088
:1034C0006EE50321002004F0ADFA4006400F606075
:1034D00066E50321002004F0A5FA4005400F606076
:1034E0005EE50321002004F09DFA4004400F606077
:1034F00056E53E4B1B7A636052E53B4B3B4A9B6D66
:103500001068984760604BE5374B384A9B6D5068B0
:103510009847606044E5374B1B68636040E5364B75
:103520001B6863603CE5314B9B7D636038E50020A0
:1035300004F0FEFF606033E52C4B1B8C63602FE5CD
:103540002E4B1B6863602BE52D4B1A78002A01D0A7
:103550000122626000221A702A4A1378002B03D0DD
:10356000022361680B4363600023137018E5264B48
:103570001B78636014E55021002004F053FAAB7807
:10358000224A9B009B58C01A606009E5174BDB6913
:10359000636005E5154B5B6A636001E5134B9B8A2D
:1035A0006360FDE40021080004F03CFAC000C00F95
:1035B0006060F5E41221002004F034FA6060EFE46A
:1035C0000A4B40331B786360EAE4084B1B7E636060
:1035D000E6E403232370E3E404232370E0E41968A2
:1035E00091430A00EAE4C04690F1FF1F84F9FF1FEF
:1035F000C8F9FF1F58F9FF1F14FAFF1F7CF9FF1FBE
:1036000081F9FF1F71F9FF1F82F9FF1F74F9FF1F76
:1036100070B5BE4CA078022800D121E1032800D16A
:103620002DE1002800D0EFE16378512B00D1DCE0E0
:1036300047D8462B00D1A0E015D8422B00D187E017
:1036400005D8412B00D17AE00322B14B75E0442B21
:1036500000D182E0452BF7D11020E178AD4B1974F1
:1036600003F098FC73E04B2B00D190E012D8472B6D
:10367000EAD12379E2781B02134314200222A54DDC
:10368000A549AB8203F0F4FCEA8AA98A287C05F0FC
:103690009FFB5CE04C2B00D185E04D2BD4D12279EF
:1036A000E37812021A4363791B041A43A3791B06B9
:1036B0001343012B4BD8974A984913730C200122CE
:1036C00043E0572B00D189E01CD8532B00D17BE07D
:1036D00000D26FE0542B00D195E0552BB4D1227964
:1036E000E178637912021B040A431A43A3791B068B
:1036F0001343012B00D987E1864B0122D9730F2098
:10370000874922E0842B00D190E00ED8832B9BD1F7
:103710002279E37812021A4363791B041A43A379CE
:103720001B0613437F4A136611E0852B00D18AE004
:10373000FF2B89D17B4BE2785C331A7007E0E2788B
:10374000744B02209A700122774903F091FC70BDFE
:103750007049E37801220B70F7E72279E3781202CF
:103760001A43637971491B041A43A37908201B0685
:103770001343684A93600422E7E72379E2781B0247
:103780001343644A6A49538212200222DDE7614DE5
:10379000E378012267490320EB7003F069FCE878C5
:1037A000FEF770FFD3E7E2785A4B63495A70012263
:1037B0001000CAE72379E2781B021343554A5F4998
:1037C000138318200222C0E72379E278514D1B02AF
:1037D0001343EB8202225A49162053E7E2784D4BFD
:1037E00058491A7104200122AFE70123494D6A7B31
:1037F0001A4204D0E2781A4201D103F025FBE178A5
:103800000D2069732CE72279E178637912021B0499
:103810000A431A43A3791B061343012B00D9F3E093
:103820003C4B012299730E2047498EE72279E378B9
:1038300012021A4363791B041A43A3791B0613432C
:10384000424A136083E72279E37812021A436379CC
:103850001B041A43A3791B061343324A536676E7C7
:103860002279E37812021A43637961781B041A43C0
:10387000A37989001B061343354A8B5067E76378A9
:10388000272B00D1ACE035D8022B00D17FE015D832
:10389000002B6BD0012B00D0D6E62279E378120200
:1038A0001A4363791B041A43A3791B061343294A5D
:1038B0005360FEF70FFE1B4BD86648E71B2B00D169
:1038C00086E01C2B00D187E0092B00D0BCE603F07A
:1038D000D7FC00286CD12379E2781B02134362796C
:1038E000A07812041343A27912061A43322104F07D
:1038F00075F82CE72B2B00D17AE02DD8E27815490A
:10390000292B73D070D94A7521E7C046DCF4FF1F1C
:1039100048F5FF1F04F0FF1F18F0FF1F10F0FF1FF6
:1039200013F0FF1F90F1FF1F06F0FF1F0CF0FF1FA9
:1039300016F0FF1F07F0FF1F05F0FF1F1CF0FF1F11
:103940001AF0FF1F08F0FF1F12F0FF1F44F5FF1FC2
:1039500054F5FF1F18FAFF1F2D2B51D04CD32E2BDF
:1039600000D071E6E278294B5A76F0E62279E378C6
:1039700012021A4363791B041A43A3791B061343EB
:10398000224A1360FEF7A6FD214B9866DFE62279F6
:10399000E37812021A4363791B041A43A3791B06C6
:1039A00013431A4A9360FEF795FD194B1867CEE64C
:1039B0002379E2781B0213436279A078120413433F
:1039C000A279810012061A43124BCB58D2188DE708
:1039D000E2780E4B1A74BAE6E2780C4B5A74B6E6EB
:1039E000E2780A4B9A74B2E6CA74B0E60A75AEE69B
:1039F000E278064B9A75AAE6E278044BDA75A6E6F9
:103A0000E278024B1A76A2E604221EE618FAFF1F9D
:103A100090F1FF1F74F9FF1F70B5214CA0780028AA
:103A20003AD1012580221F4B120518701E4B290028
:103A300018701E4B1D7004F033F84422A0781C4B04
:103A400042439B18DB7D2A00002B00D0022220215C
:103A500003F0C4FF80220721A078520504F020F86B
:103A60002379E0781B0203436079A57800040343BF
:103A7000A079AA00000618430E4B9B185B6F98476D
:103A800024210200280003F0A9FF8022A07812055B
:103A9000012104F012F870BD0422074B1A70FAE7F6
:103AA000DCF4FF1F81F9FF1F71F9FF1F72F9FF1F7F
:103AB00084F9FF1F90F1FF1F48F5FF1F70B5224CDE
:103AC000A07800283BD101258022204B12051870D8
:103AD0001F4B290018701F4B1D7003F0E1FF44229B
:103AE000A0781D4B42439B18DB7D2A00002B00D0A1
:103AF0000222202103F072FF80220721A0785205C4
:103B000003F0CEFF2379E0781B0203436079A578A8
:103B100000040343A079AA00000618430F4B40425B
:103B20009B185B6F984724210200280003F056FF82
:103B30008022A0781205012103F0BFFF70BD04228E
:103B4000074B1A70FAE7C046DCF4FF1F81F9FF1F2C
:103B500071F9FF1F72F9FF1F84F9FF1F90F1FF1F1A
:103B600048F5FF1FF8B52421002003F05BFF002378
:103B7000414C424E424D206533702B7E002B51D17B
:103B8000404B6367A365A367E36728210020E76FC5
:103B900003F048FFB8472921E8620020E76F03F0EF
:103BA00041FFB8472A2128630020E76F03F03AFF5E
:103BB000B8472B2168630020E76F03F033FFB84755
:103BC0002C21A8630020E76F03F02CFFB8472421C5
:103BD000E863002003F026FF00232B4A20651370C2
:103BE0002A4A180013602A4A2A4F13602A4A33705F
:103BF000136022004C32137080226364D200D91902
:103C0000043308609342FAD1244EB37B002B11D1C8
:103C1000F37B002B1ED0337B002B2AD001234034B2
:103C20002370F8BD1E4B63671E4BA3651E4BA36735
:103C30001E4BA9E7D825AD001D4B2800E9181D4BE8
:103C40000422C91803F0AAFAEC2304359B009D4214
:103C5000F2D1DDE7A025AD00174B2800E91879184F
:103C6000042203F09BFAD82304359B009D42F3D134
:103C7000D1E74034D4E7C04690F1FF1F72F9FF1F2F
:103C800084F9FF1F717D000010F2FF1F3CF5FF1F3C
:103C900050F5FF1F54F5FF1FE4F4FF1F04F0FF1F52
:103CA000617D0000697D0000657D00006D7D000084
:103CB000A4FCFFFFE8F4FF1F80FDFFFF70B5442563
:103CC0004543584E584B7519EA6A04009A420CD87D
:103CD0002A6B9A4209D86A6B9A4206D8AA6B9A4212
:103CE00003D8EA6B9A4200D871E04425654302226A
:103CF00075190021200003F0D3FEE86A05F016FED6
:103D000007F0CAFB0022494B06F09AFDA222484B5D
:103D1000120606F061F907F049FB28210200200095
:103D200003F05CFE286B05F001FE07F0B5FB0022F6
:103D30003E4B06F085FDA2223D4B120606F04CF9E3
:103D400007F034FB29210200200003F047FE686BD6
:103D500005F0ECFD07F0A0FB0022344B06F070FDEF
:103D6000A222334B120606F037F907F01FFB2A2177
:103D70000200200003F032FEA86B05F0D7FD07F02B
:103D80008BFB0022294B06F05BFDA222284B12067A
:103D900006F022F907F00AFB2B210200200003F0B5
:103DA0001DFEE86B05F0C2FD07F076FB00221F4BFD
:103DB00006F046FDA2221E4B120606F00DF907F092
:103DC000F5FA02002C21200003F008FE70BD02224B
:103DD000002103F072FE174EA300F618B36FE86AD5
:103DE000984728210200200003F0F8FDB36F286BEC
:103DF000984729210200200003F0F0FDB36F686BA3
:103E000098472A210200200003F0E8FDB36FA86B59
:103E100098472B210200200003F0E0FDB36FE86B10
:103E20009847CEE784F9FF1FFFFF3F0000004042A4
:103E3000941AED4290F1FF1F73B5034CA378002B49
:103E400000D091E102E0C046DCF4FF1F607805F08D
:103E5000DBF9EB0105023C02520265029202A2026A
:103E6000C1020908090809080908D202F0020E0374
:103E70003303460356036603790389039C03AC03AB
:103E8000BB03CA03D903E803F703060424040908A3
:103E9000090809083B045304090809080908090826
:103EA000090809080908090809080908090809088A
:103EB000090809080908090809080908090809087A
:103EC000090809080908090809080908090809086A
:103ED000090809080908090809080908090809085A
:103EE000090809080908090809080908090809084A
:103EF000090809080908090809080908090809083A
:103F00000908090809080908090809080908090829
:103F10000908090809080908090809080908090819
:103F2000090809080908090809086B047C048D04BC
:103F3000A004B904CA04D704E404F60411052B054F
:103F4000450557056905090809087B058D059F0585
:103F5000AD050908C0050908090809080908D605BA
:103F60000908E805FD051206090809082E0640069D
:103F70005206640609080908090809080908090819
:103F800009080908090809080908090809080908A9
:103F9000090809080908000105010A010F011D01AE
:103FA0002B01300135013A013F01440149014E0125
:103FB0000908090809080908530109085801680196
:103FC00009088F0194019901BC01DC010908090865
:103FD0000908090876067B068C06090809080908FD
:103FE00009089D06AB06BA06E101E60109080908C1
:103FF000090809080307400709086D0709087F0732
:104000000908090809080908090809080908090828
:104010000908090809080908090809080908090818
:104020000908090809080908090809080908090808
:1040300009080908090809080908090809080908F8
:10404000090809080908090893070908AB07BB070D
:10405000E007E178002004F06BFB73BDE1780020FD
:1040600004F0E4FBF9E7E178002004F00BFCF4E74E
:10407000002004F09FFCE178002803D1A07804F030
:1040800047FCEAE7A07804F013FCE6E7002004F020
:1040900091FCE178002803D1A07804F039FBDCE73B
:1040A000A07804F021FCD8E7E178002004F020FBA0
:1040B000D3E7E178002004F00BFDCEE7E1780020A3
:1040C00004F0BBFCC9E7E178002004F0CBFCC4E7B6
:1040D000E178002004F0A1FCBFE7E178002004F0C3
:1040E000D5FCBAE7E178002004F008FDB5E7E178F7
:1040F000002004F0DBFCB0E7E178002004F00CFCC9
:10410000ABE72379E0781B020343607900040343A3
:10411000A07900061843DE4B5B6F9847DD4B1861B2
:104120009BE72179E07809020143607900040143AB
:10413000A0790006084317D4D64B1B7E012B01D073
:1041400003F012FE002809D00100D34805F066F8FC
:1041500014210200A07804F05DFA7EE7A078CF4A2F
:10416000142104F057FA78E70422CD4B1A7074E753
:10417000E178002004F070FB6FE7E178002004F0A4
:10418000EBFA6AE72179E0780902014360790004DB
:104190000143A07900060843E6D4BE4B1B7E012BE9
:1041A00001D003F0E1FD002809D00100BA4805F074
:1041B00035F813210200A07804F02CFA4DE7A0781E
:1041C000B64A132104F026FA47E7E178002004F00C
:1041D00037FD0021A07804F04BFA2379E1781B0227
:1041E0000B436179020009040B43A179A078090609
:1041F00019430423002904D01A43002104F00AFAC9
:104200002BE79A4304F006FA27E7E178002004F050
:1042100029FD22E7E178002004F0D2FC1DE7E178D7
:10422000002004F0B9FC18E79E4BE2781878237957
:104230001B021343627912041343A27912061A4334
:10424000002803D1372103F0C9FB06E7964B37213D
:104250001B680020D21803F0C1FBFEE6914B1878D2
:1042600000280DD12379E2781B02134362792121C2
:1042700012041343A27912061A4303F0AFFBECE6D3
:104280002121002003F0CEFB2279E37812021A43A9
:10429000637950211B041A43A3791B061343C01AE8
:1042A000814B1860A578280003F0BCFB2279E378E5
:1042B00012021A436379AD001B041A43A3791B064B
:1042C0001343C01A794BE850C7E60122784BE078D7
:1042D0001A7023791B020343607900040343A07919
:1042E000000618436A4B5B6F9847242102000020A8
:1042F00003F074FBB1E62379E0781B020343607995
:1043000000040343A07900061843614B5B6F984794
:1043100022210200002003F061FB9EE62379E07871
:104320001B02034360795A4D00040343A079000641
:1043300018436B6F9847C317C01858402865A0787A
:10434000202103F06FFB430700D486E62379E07851
:104350001B0203436079A67800040343A07900069A
:104360001843B300ED186B6F98472421020030000A
:1043700003F034FB71E62279E37812021A43637981
:1043800000201B041A43A3791B061343414AD3623E
:10439000FFF794FC61E6434AE1783E4B107859728E
:1043A000002808D19A7A9B7D009101930621030091
:1043B00003F0ECFA51E61021002004F059F9E278FC
:1043C0003C4BD2081840120202431021002004F096
:1043D00021F942E63349E2782E4B08789A72002898
:1043E00000D03AE6997D01915B7A062100930300A3
:1043F00003F0CCFA31E60121002003F013FB0A237D
:10440000020021799A43E3780902194363791B0476
:104410001943A3791B060B430221D80700D50A4391
:104420000B4201D008231A43A078012103F0D6FAE9
:1044300013E60121002003F0F5FA0523020021799B
:104440009A43E3780902194363791B041943A3795A
:104450001B060B4301210B4200D00A439B0701D5E9
:1044600004231A43A078012103F0B8FAF5E5227974
:10447000E37812021A4363791B041A43A3791B06DB
:104480001343012B00D96FE6024AD375E5E5C04618
:1044900090F1FF1F84F9FF1F0024F400B500100005
:1044A00048F5FF1FC8F9FF1F60F9FF1F74F9FF1FD0
:1044B00072F9FF1FFFE0FFFF2379E0781B0203433F
:1044C000607900040343A07900061843E54B5B6F55
:1044D000984725210200002003F080FABDE52279EB
:1044E000E37812021A43637900201B041A43A3796C
:1044F0001B061343DC4A5363FFF7E0FBADE522796B
:10450000E37812021A43637900201B041A43A3794B
:104510001B061343D44A1363FFF7D0FB9DE52379B1
:10452000E0781B020343607900040343A07900068E
:104530001843CC4B5B6F984727210200002003F003
:104540004DFA8AE52279E37812021A436379002052
:104550001B041A43A3791B061343C34A9363FFF753
:10456000ADFB7AE52379E0781B0203436079000410
:104570000343A07900061843BA4B5B6F9847262186
:104580000200002003F02AFA67E52279E37812029C
:104590001A43637900201B041A43A3791B061343B3
:1045A000B14AD363FFF78AFB57E52379E2781B0210
:1045B000134362792D2112041343A27900201206BD
:1045C0001A4303F00BFA48E52379E2781B02134300
:1045D00062792E2112041343A279002012061A4395
:1045E00003F0FCF939E52379E2781B021343627981
:1045F0002F2112041343A279002012061A4303F05C
:10460000EDF92AE52379E2781B0213436279302120
:1046100012041343A279002012061A4303F0DEF9B4
:104620001BE52379E2781B021343627933211204DC
:104630001343A279002012061A4303F0CFF90CE5C8
:104640002379E2781B021343627934211204134365
:10465000A279002012061A4303F0C0F9FDE40121FB
:10466000002003F0DFF9C023020021799A43E378A8
:104670000902194363791B041943A3791B060B43F1
:10468000D90701D540210A439B0701D580231A434E
:10469000A078012103F0A2F9DFE40121002003F05A
:1046A000C1F9724AE37810402279012112021343C2
:1046B000627912041A43C02312029B001A4002437B
:1046C000A07803F08BF9C8E410250121002003F045
:1046D000A9F92179E3780902194363790200AB4013
:1046E0001943A379AA431B060B4300D02A43A078A1
:1046F000012103F073F9B0E40121002003F092F9E5
:10470000202502002179E378090219436379AA433D
:104710001B041943A3791B060B4300D02A43A0783E
:10472000012103F05BF998E42379E2781B0213433B
:104730006279602112041343A279002012061A4301
:104740004B4B5A6003F04AF987E42379E2781B0265
:1047500013436279612112041343A27900201206E7
:104760001A43434B9A6003F039F976E4E278404B00
:104770001C211A73002003F055F92279E378120204
:104780001A43C0B2120402431C21A07803F026F998
:1047900063E42379E2781B021343354A1C21D38159
:1047A000002003F03FF92279E37812021A43FF2335
:1047B000D2051B041840D20D02431C21A07803F03F
:1047C0000DF94AE42379E2781B02134362795921F7
:1047D00012041343A279002012061A43244B1A61D3
:1047E00003F0FCF839E4E178214A1175937D0191D9
:1047F000527D062100920022100003F0C7F82CE43D
:10480000E1781B4A5175937D127D0091019200223F
:104810000621100003F0BAF81FE42379E2781B02A6
:10482000134362795A2112041343A279002012061D
:104830001A430F4B1A6203F0D1F8FFF70EFC2379ED
:10484000E2781B02134362795B2112041343A279BD
:10485000002012061A43064B5A6203F0BFF8FFF716
:10486000FCFBC04690F1FF1F84F9FF1FFFFCFFFF18
:10487000C8F9FF1F2379E2781B02134362791204FF
:104880001343A27912061A43EE4BD1B29A62120A6E
:10489000D2B2DB6A009200220191DBB25D211000EE
:1048A00003F074F8FFF7D9FB2279E37812021A4378
:1048B00063791B041A43A3791B061343E14AD362AD
:1048C000926ADBB2D1B2120AD2B2009200220191F6
:1048D00010005D2103F05AF8FFF7BFFB2379E2785F
:1048E0001B02134362795E2112041343A279002054
:1048F00012061A43D34B1A6303F070F8FFF7ADFBAF
:104900002379E2781B0213436279182112041343BE
:10491000A279002012061A43CA4B9A6103F05EF88E
:10492000FFF79BFB2379E2781B021343627919217D
:1049300012041343A279002012061A43C14BDA6114
:1049400003F04CF8FFF789FB2379E2781B0213434D
:1049500062795C2112041343A279002012061A43E3
:10496000B84B5A6303F03AF8FFF777FB2379E27804
:104970001B02134362795F2112041343A2790020C2
:1049800012061A43AF4B9A6303F028F8FFF765FB52
:10499000AC4AE378117D93750191527D0621009216
:1049A0000022100002F0F2FFFFF757FB2279E178B6
:1049B000637912021B040A431A43A3791B061343AB
:1049C000022B01D9FFF7D0FB9F4B54331970FFF72F
:1049D00044FB2279E37812021A4363791B041A43D9
:1049E000A3791B061343974A012B04D197491370EF
:1049F0000B70FFF732FB00231370FFF72EFB2379B8
:104A0000E2781B0213436279522112041343A27904
:104A1000002012061A438B4BDA6302F0DFFFFFF728
:104A20001CFB8849E0780B00403318704423CB18F6
:104A30004A6C1B78413101900978120A0091D2B278
:104A40006321002002F0A2FFFFF707FB7D49E07819
:104A50000B004133187044234A6CCB18403109785D
:104A6000120A1B78D2B2019100906321002002F05B
:104A70008DFFFFF7F2FA734923790800E2781B02F1
:104A800013436279403012041343A27912061A4389
:104A90004A640078413101900978D3B2120A00913A
:104AA000D2B26321002002F071FFFFF7D6FA23791A
:104AB000E2781B0213436279032112041343A279A3
:104AC000009112061A430023180003F003F8FFF7C1
:104AD000C4FA03212379E2781B0213436279002090
:104AE00012041343A279009112061A43042302F020
:104AF000F1FFFFF7B2FA03212379E2781B02134397
:104B00006279002012041343A279009112061A431D
:104B1000082302F0DFFFFFF7A0FA03212379E278F0
:104B20001B0213436279002012041343A2790091FF
:104B300012061A430C2302F0CDFFFFF78EFAE2783B
:104B4000434B1A72FFF789FA2379E0781B0203437B
:104B5000607900040343A079000618433A4B5B6F69
:104B600098473B4B1860FFF778FA2379E0781B02EF
:104B70000343607900040343A07900061843324BD5
:104B80005B6F9847324B5860FFF767FAE178304B1C
:104B900099759A7A01915B7A062100930023180097
:104BA00002F0F4FEFFF759FA2379E1781B020B4378
:104BB0006179002009040B43A1790906194303F028
:104BC0005DFCFFF74AFA2379E2781B02134362790E
:104BD0001F4D12041343A27912061A432B8C9A42DA
:104BE00001D1FFF73AFA174B1878002824D10C238B
:104BF00044262A840A2192B20093083B02F06AFFFD
:104C00003300A07854214343EB18DA69D317D21844
:104C10005A4002F0E3FE8022A07892054643AD1987
:104C2000EB690721002B03DA02F03AFFFFF715FAD0
:104C300002F043FFFFF711FA0622064B1A70FFF746
:104C40000CFAC046C8F9FF1F90F1FF1F72F9FF1F51
:104C500084F9FF1F48F5FF1F854B864E1D78002DF8
:104C600024D05021002002F0DDFE2279E3781202E8
:104C70001A43637921211B041A43A3791B061343AA
:104C8000C01A3060A578280002F0CCFE2279E378C3
:104C900012021A436379AD001B041A43A3791B0661
:104CA0001343C01A744BE850FFF7D7F92379E27821
:104CB0001B0213436279502112041343A279280086
:104CC00012061A4302F08AFEA3789B00F550FFF704
:104CD000C4F92379E2781B0213436279674D120409
:104CE0001343A27912061A43EB699A4201D1FFF7E6
:104CF000B4F95F4B187800289ED1D317EA61D21817
:104D00005A40542102F06AFE44238022A078920582
:104D10004343ED18EB690721002B03DA02F0C0FED4
:104D2000FFF79BF902F0C9FEFFF797F92379E278C4
:104D30001B0213436279532112041343A27900200A
:104D400012061A434D4B5A6202F048FEFFF785F9EE
:104D50002379E2781B02134362791521120413436D
:104D6000A279002012061A43444B9A82444B5A43BC
:104D700002F034FEFFF771F980222379E0781B02FC
:104D800003436079520500040343A07900061843E9
:104D900005D00021080002F083FEFFF75EF9010054
:104DA00002F08BFEFFF759F92379E2781B021343D7
:104DB0006279122112041343A279002012061A43C9
:104DC00002F00CFEFFF749F92379E5781B022B432B
:104DD00065792A4E2D042B43A5792D061D430BD151
:104DE00029002800FDF72AFE4423A2785343F31834
:104DF00040331D70FFF731F901210020FDF71EFE41
:104E00004423A27853430122F31840331A70FFF76A
:104E100024F92279E37812021A4363791B041A43B6
:104E2000A3791B06134306D0012B0ED00422154B89
:104E30001A70FFF712F9114A1376134B134A5A6787
:104E40009A659A67DA67FFF708F90C4A13760E4BF2
:104E50000F4A5A670F4A9A650F4A9A670F4ADA67EC
:104E6000FFF7FBF80322074B1A70FFF7F6F8C0466E
:104E7000C8F9FF1F74F9FF1F60F9FF1F84F9FF1FB6
:104E80000071020048F5FF1F90F1FF1F717D0000C7
:104E9000617D0000697D0000657D00006D7D000082
:104EA0006423F7B5B84CB94D22782B706A7021791C
:104EB000E3780902194363791B041943A3791B069C
:104EC0000B436B60292A01D101F02AF900D9EFE0E8
:104ED000162A01D100F0DBFD69D80A2A00D12CE2A4
:104EE00018D8042A00D11FE20AD8022A00D1FAE118
:104EF00000D9FBE1012A00D1F2E102232B70F1E19C
:104F0000062A00D116E200D211E2092AF5D1FEF7F5
:104F10007FFBE7E10E2A00D120E31AD80C2A01D149
:104F200000F0E9FC01D800F0D2FCA078002800D005
:104F3000F7E16378012B01D100F0C0FC002B01D117
:104F400000F0B2FC022B01D100F0BBFC03232B705C
:104F5000C8E1132A01D100F0E2FC0ED80F2ACCD10F
:104F6000A378012B00D133E3002B00D117E3022BF0
:104F700000D131E304232B7017E3142A01D100F090
:104F800007FD152AB9D160780C2800D9AAE1804A1A
:104F900004F03AF9200527052E0535053C054305A3
:104FA0004B0552055905600567056E057505202AF4
:104FB00001D100F01DFC3DD81A2A01D100F0FEFFFE
:104FC0000FD8182A01D100F076FD01D800F063FD5A
:104FD00063782E2B01D900F0E8FF01216D4AD154EE
:104FE00080E11C2A01D100F04AFE01D200F072FDDE
:104FF0001E2A00D17AE31F2A00D07EE760781428A9
:1050000000D9BAE2A378002B00D0ACE3624B800059
:10501000C158624B69601B78002B00D162E1604B84
:10502000082219605A4B002900D098E319680A43F6
:105030001A6057E1242A01D100F07CFE12D8584DA5
:10504000222A01D100F06AFE01D800F01EFE2A7863
:10505000E2706A782271AA786271EA78A271FEF72A
:10506000D7FA3FE1262A01D100F0C4FF01D200F0B7
:10507000B6FF272A01D100F08CFE282A00D03CE799
:10508000FF2B00DD2EE160780B2801D901F044F8F8
:10509000444D9B0004F0B8F8D107D907E107E907B0
:1050A000F207FB0703080B0813081A082008280852
:1050B000452A00D1A4E200D986E0332A01D101F0CB
:1050C0005EFA49D82D2A01D101F0D1F91DD82B2A39
:1050D00001D101F009F901D801F090F860780B28AE
:1050E00001D901F0C0F9A3782E4A2F4D9B0004F09E
:1050F0008BF868096E0974097A09810988098E0993
:1051000094099A099F09A309A909302A01D101F03C
:1051100014FA0ED82E2A00D0EFE6214B1978E17050
:10512000597821719978DB786171A371FDF7FCFCE6
:10513000D8E0312A01D101F014FA322A00D0DCE69D
:10514000174B1978E170597821719978DB78617182
:10515000A371FEF7B3FCC5E0402A00D144E225D894
:10516000382A01D101F018FA392A01D101F02EFABA
:10517000372A00D0C1E60C4A1268FF2A00D9B1E0F4
:10518000084992005350ADE0DCF4FF1F48F5FF1FC3
:10519000E4F4FF1F42FAFF1FE8F4FF1F40F5FF1F72
:1051A0003CF5FF1F54F5FF1F50F5FF1F422A00D1A9
:1051B00020E200D21BE2432A00D11EE2442A00D0A2
:1051C0009BE602F0DEFB8DE0852A01D100F021FE96
:1051D00042D8802A01D100F0EDFD1ED8472A00D127
:1051E00014E200D20FE2502A00D086E6A2498A6C6F
:1051F000072A77D860780C2874D8A04C04F004F8FB
:10520000F309020A110A200A2F0A4A0A5A0A690AED
:10521000780A870A960AA50AB40A822A01D100F000
:10522000EAFD01D200F0CCFD832A01D100F0E9FDB6
:10523000842A00D061E6924A527B920701D500F0A1
:10524000E4FD904A934200D96BE004218A4A40323F
:1052500011708D4A536345E0892A00D130E213D89A
:10526000872A01D100F02AFE01D800F0D8FD63782A
:10527000012B00D1DDE1002B00D1CAE1022B00D1CE
:10528000DFE103232B702DE08D2A01D100F047FED2
:1052900019D88A2A00D030E662787C4B002A00D0E8
:1052A00013E31A70E3787A4A1370774A1178794ACF
:1052B0001170002278490A7078490A70784A11788A
:1052C0000B4313700EE0F22A00D1CCE1FF2A00D08C
:1052D00013E6744A934205D101226B4BDA7201E066
:1052E000FEF79AFBF7BDFEF7E9FBFBE7A078002885
:1052F00017D103F071F844210122A0786A4B414391
:105300001A546A4B5B18DB7D002B08D1202102F078
:1053100065FBA0780022242102F060FBE2E7022274
:10532000F4E704232B70DDE7FDF7FEFBDAE7FEF779
:1053300083FDD7E7FDF71EFDD4E7A378022B00D14C
:1053400094E0032B00D1BFE0002B00D000E1637894
:10535000522B6BD022D8462B5FD00ED8422B56D082
:1053600004D8412B3FD003232B703FE0442B51D076
:10537000452BF8D1424B1B7C37E04C2B53D006D841
:10538000472B4DD04B2BEED13D4BDB782DE04D2BF9
:1053900052D0512BE7D13A4B5B7B26E0802B54D087
:1053A00009D8542B4BD044D3552B4BD0572BDAD1A3
:1053B000334B1B7919E0832B52D006D8812B47D071
:1053C000822BD0D12C4B5B6C0FE0842B4BD0852BE8
:1053D000C9D1294A364B516E4B4336495B18536647
:1053E0005B005B0801E0264B9B786B60324B1B78BF
:1053F000002B00D176E7314B6968082219601F4BFA
:10540000002900D0A6E019680A431A606AE71C4B1D
:105410001B78EAE71A4B9B68E7E7194B5B8AE4E7DE
:10542000174B9B8AE1E7164B5B78DEE7144B1B8B2F
:10543000DBE7134BDB8AD8E7114B1B7BD5E7104B1F
:105440009B7BD2E70E4BDB7BCFE70B4B4033DFE799
:10545000094B40331B78043B594259416960C5E709
:10546000054B1B6EC1E7164B1B68BEE76378154AF8
:105470009B009B58B9E7C04690F1FF1FE4F4FF1F63
:1054800004F0FF1FFF07000010F2FF1F5CF9FF1F71
:1054900078F9FF1F3EFAFF1F73F9FF1F71FAFF1F14
:1054A0005DF9FF1FD204000072F9FF1F84F9FF1F8E
:1054B0006D4EC6413930000040F5FF1F3CF5FF1F1F
:1054C00044F5FF1F54F5FF1F6378272B30D014D805
:1054D000022B26D007D8002B21D0012B00D042E789
:1054E000B04B5B6881E71B2B1DD01C2B1DD0092BFB
:1054F00000D038E7AB4BDB6877E72B2B1FD005D804
:10550000A84A292B19D016D9537D6EE72D2B1CD014
:1055100018D32E2B00D026E7A24B5B7E65E7A14B6C
:10552000A2E7A04B77E79F4B25E79E4B5B7C5CE7B0
:105530009C4B9B7C59E7D37C57E7137D55E7994BF0
:105540009B7D52E7974BDB7D4FE7964B1B7E4CE7ED
:10555000042309E7196891431960C3E6A278002A79
:1055600004D0022A0CD004232B70BBE66278002AF8
:1055700003D11800FDF78FF9B4E603232B70B1E6D1
:105580006078FF2807D0002B02D1FDF709F9A9E6C2
:10559000FDF714F9A6E61800FDF75AF9A2E66078BF
:1055A000FF2812D0FDF718F968607F4B1B78002B9D
:1055B00000D197E67D4B6968082219607C4B002971
:1055C0000ED119680A431A608CE6FDF753F9EBE730
:1055D0006078FDF781F9E7E76078FDF727F9E3E701
:1055E0001968914319607DE602F07AF97AE602F0D3
:1055F000C5F977E602F0C3F974E602F0C1F971E685
:1056000002F0C0F96EE602F0BEF96BE602F0BCF9FA
:1056100068E60121674A5170674902324978117082
:1056200066490868591CC35C8B540B000829F9D1E2
:1056300058E604226B711023EA71CB32AA712B71E8
:1056400050E6012380215B4A890153705A4B023294
:105650005B7813705A4B5B481C781818013314544C
:105660008B42F8D13EE66378812B00D03AE6A378EE
:10567000922B00D036E6A379A32B00D032E66379D3
:10568000B42B00D02EE62379C52B00D02AE6E37890
:10569000D62B00D026E680224B4B5A6072B60022F1
:1056A0004A4B4B491A6001234A4A5B42D367C022E6
:1056B00052008B50484A494B1A60FCF7F3FF11E641
:1056C0006278002A00D00DE6A278002A00D009E610
:1056D000434A934200D005E600230422694641482C
:1056E000009301F0C5FCFCF7DDFFFBE560781428B2
:1056F00000D942E7A278002A13D13B4A81008B509F
:105700002D4B9B7B002B00D1ECE5002800D1E9E577
:10571000364BD7308000C1188918042201F0A8FC4C
:10572000E0E5FF2A00D0FCE52F4C00280ED1D8255B
:10573000EC26AD00B6002D4B2800E91861180422B4
:10574000043501F095FCB542F5D1CBE5274BD730B8
:105750008000C1186118042201F08AFCC2E51968B2
:1057600091431960BEE5FF2B00D0DAE51E4C0028FE
:105770000ED1D825EC26AD00B6001C4B2800E91848
:1057800061180422043501F009FDB542F5D1A9E5FF
:10579000164BD7308000C1186118042201F0FEFCBE
:1057A000A0E5C04618FAFF1F40F5FF1F3CF5FF1F9C
:1057B000E4F4FF1F10F2FF1F04F0FF1F00F0FF1FB3
:1057C000F81F000009E0FFFF40F00F4010E000E08C
:1057D00000E100E004E100E07856341200F0FF1F21
:1057E000D2040000FE070000E8F4FF1FA4FCFFFF46
:1057F0006678142E00D9C0E6A07843B2002B27DAD1
:10580000C30706D52121002002F00CF9C24AB600D8
:10581000B050C24B1B78002B07D06378BE49C04AFA
:105820009B0058581268821A5A50BE4B9B7B002B23
:1058300000D157E56078002800D153E5BA4BD73046
:105840008000C118B44B0422C91801F011FC49E5CD
:10585000002800D065E5212102F0E4F84C23AE4990
:10586000B6007050A578AD4A6B439B5C002B08D006
:105870006278AB4BAA189200A800C3585058C31ABC
:105880005350A84B9B7B002B00D12BE56078002860
:1058900000D127E54219D7309200401989188000BD
:1058A000042201F0E5FB1DE59C4B1878002802D18D
:1058B00002F088FD16E506232B7013E502F08CFD3F
:1058C00010E502F093FD68600CE50122E9E4A3789D
:1058D000022B0DD16078372800D94EE6934BA030CB
:1058E0008000C118924B0422C91801F0C1FBF9E4F1
:1058F00004232B70F6E4A378022B0DD160783728AF
:1059000000D93AE6894BA0308000C118884B0422A8
:10591000C91801F043FCE5E404232B70E2E460784D
:10592000844C092815D803F065FC05090C0F1D23CC
:1059300026292C072268D31823600AE02268D31A8C
:10594000FAE722685343F7E72068190003F0F0FCF8
:1059500020602168784B0822002915D119680A4374
:105960001A60BFE42068190003F0C8FD2160F0E769
:1059700022681340E0E722681343DDE722685340C2
:10598000DAE72368DB43D7E7196891431960A9E494
:10599000684A1168684A8B420CDA032310689843FE
:1059A000013303431360082300290FD111680B430F
:1059B000136097E48B4204D1062310689843053B9B
:1059C000EFE7052310689843033BEAE71168994322
:1059D000116087E41268120700D483E4574A5364C5
:1059E00080E41268120700D57CE4544A536479E4D9
:1059F0001268D20700D475E4504A536472E4126806
:105A0000D20700D56EE44D4A53646BE41268520726
:105A100000D467E4494A536464E4116805221142E2
:105A200000D15FE4454A53645CE41268920700D4F5
:105A300058E4424A536455E41268920700D151E495
:105A40003E4A53644EE41268D20600D44AE43B4A0C
:105A5000536447E41268920600D443E4374A53641F
:105A600040E41268520600D43CE4344A536439E4FA
:105A70001268120600D435E4304A536432E41268E6
:105A8000D20500D42EE42D4A5364FFF72BFC2B4A99
:105A90005364FFF727FC29498A6C072A01D9FFF7CD
:105AA00021FC501C8864264892008218486C4B6484
:105AB000D060FFF717FC214A936C002B01D1FFF750
:105AC00011FC013B1E4993649B00CB18DB685364B7
:105AD000FFF708FC194D2A004C321278002A0ED12B
:105AE000174E0A32591C13D1124B1B685A43F262EB
:105AF000FCF7F0FC2B0001224C3330631A70607805
:105B0000032801D9FFF7EEFB03F074FB1C315E8B19
:105B10005343F362ECE7C046E8F4FF1FC8F9FF1FE8
:105B200060F9FF1F04F0FF1FA4FCFFFF80FDFFFFD3
:105B300054F5FF1F3CF5FF1FE4F4FF1F90F1FF1F1A
:105B400010F2FF1FFCF7C6FCD34B1A6BDB6A801AFE
:105B5000C21780185040984204D900234C352B704E
:105B6000FFF7C0FB6B6C013B6B64FFF7BBFBA078DE
:105B70000F2101F057FF0124044009D00023C74A38
:105B80004C3511682B70103399431160FFF7AAFB55
:105B9000C14EF36A002B12D0FCF79CFC336BC31A86
:105BA000DA179B185340F26A934208D91023BB4A74
:105BB0004C3511682C700B431360FFF793FB6B6C33
:105BC000013B6B64FFF78EFBA0780F2101F02AFFE9
:105BD0008024044009D00023B04A4C3511682B7052
:105BE000103399431160FFF77DFBAB4EF36A002B36
:105BF00012D0FCF76FFC336BC31ADA179B185340B3
:105C0000F26A934208D91023A44A4C3511682C70CB
:105C10000B431360FFF766FB6B6C013B6B64FFF794
:105C200061FBA0780F21802401F0FCFE6400044099
:105C300009D00023994A4C3511682B7010339943D1
:105C40001160FFF74FFB944EF36A002B12D0FCF764
:105C500041FC336BC31ADA179B185340F26A934224
:105C600008D910238D4A4C3511682C700B431360F2
:105C7000FFF738FB6B6C013B6B64FFF733FB0022D3
:105C8000874B40331A70FFF72DFB60780A280CD839
:105C9000844B03F0AFFA0614181C22282C30343839
:105CA0003A001B682A68D3182B6029687B4B0822AE
:105CB00000292ED119680A431A60FFF713FB1B68ED
:105CC0002A68D31AF0E71B682A685343ECE7286870
:105CD000196803F02DFB2860E7E72868196803F0CE
:105CE0000DFC2960E1E71B682A681340DCE71B68AC
:105CF0002A681343D8E71B682A685340D4E71A6818
:105D0000D2431A60D1E72A68FBE719682A6829603C
:105D1000F7E7196891431960FFF7E4FA2A78E2700F
:105D20006A782271AA786271EA78A271FEF784F823
:105D3000FFF7D8FA6078052801D9FFF7D3FA574B57
:105D400003F058FA03090F151B210F2219680A40A6
:105D50001A60FFF7C7FA1022196891431960FFF71C
:105D6000C1FA2022196891431960FFF7BBFA40225B
:105D7000196891431960FFF7B5FA802219689143B9
:105D80001960FFF7AFFA1968474A0A401A60FFF72F
:105D9000A9FAA378002B01D0FFF7C3FA6378142B7C
:105DA00001D9FFF7EAFB414A9B001168404A99502C
:105DB000FFF798FA00223A4B40331A70FFF792FA35
:105DC0006278002A05D0012A09D003232B70FFF73F
:105DD00089FA0122324B40331A70FFF783FA3549B2
:105DE0008B4201D9FFF79DFA2D490800403002701F
:105DF0004B64FFF777FA0222294B40331A70FFF702
:105E000071FAFCF765FEFFF76DFA08232B70FFF7B8
:105E100069FA0022224B40331A70FFF763FA01251A
:105E20001D49254A4D7050788C1C8870214883424A
:105E300026D8567B2A002E4023D11800694600F050
:105E4000C1FF6B461B7863706B465B78A3706B4633
:105E50009B78E3706B469B7923716B465B7963712A
:105E60006B461B79A3716B46DB782672E371295D63
:105E7000227A013552182272082DF8D1FFF732FA32
:105E80002A008B1C0021D1540132082AFBD11A7838
:105E90001A72FFF727FAC04610F2FF1FE4F4FF1F43
:105EA00090F1FF1F50F5FF1FFFFEFFFF3CF5FF1FA6
:105EB000E8F4FF1FFF07000004F0FF1F60780328CD
:105EC00001D9FFF70FFA03F095F902112025DE4BF7
:105ED0001A004C331B784032AB71DC4B12785B6B91
:105EE000EA711A0A6A712B71FFF7FCF9D64B1A0096
:105EF00040321278EA711A004C3212785B6CAA7147
:105F00001A0A6A712B71FFF7EDF9D14B1B686B60B0
:105F1000FFF7E8F9CF4B1B686B60FFF7E3F9607898
:105F200003283ED803F066F917022E39C74C002229
:105F30002500A16B3C358A4201D1FFF7D3F99000CF
:105F400046599E421CD1230001393C338A4211D369
:105F5000A163FFF7C7F9BD4A916B092906D8481C10
:105F6000890090635218D363FFF7BCF909232B70A3
:105F7000FFF7B8F91D186D680132C5500430E5E728
:105F80000132D8E700231900B04A93633C3299509C
:105F90000433282BFBD1FFF7A5F90A236B60FFF729
:105FA000A1F903232B70FFF79DF9FF2B01D0FFF719
:105FB000E4FA0122A84B1A70FFF794F963782E2BAC
:105FC00004D80021A54AD154FFF78CF9FF2B01D04A
:105FD000FFF7D3FA0022A04B1A70FFF783F962781B
:105FE0002E2A01D9FFF7C9FA9B4992008A185360FB
:105FF000FFF778F9954B964A596E186F1160996EB4
:10600000944A1160D96E904A516495494C320860A7
:1060100074215918097811709A6F1A63DA6FDA626D
:1060200064331B7F8D4AD15C002901D00121D154FA
:106030000022894B5A70FFF755F9A278EB5892006D
:10604000A958CB18AB50FFF74DF9A278EB58920046
:10605000A958CB1AAB50FFF745F9A278EB5892003C
:10606000A9584B43AB50FFF73DF9A478E958A40079
:10607000285903F05DF92851FFF734F9A478E9585D
:10608000A400285903F03AFA2951FFF72BF9A27816
:10609000EB589200A9580B40AB50FFF723F9A278B8
:1060A000EB589200A9580B43AB50FFF71BF9A278AD
:1060B000EB589200A9584B40AB50FFF713F9EB583F
:1060C000A278DB439200AB50FFF70CF9EA58A378B3
:1060D0009B00EA50FFF706F9A278E8589200A95809
:1060E000A850E950FFF7FEF8A278EB589200AA58A2
:1060F0009A4200DCABE1032359490A689A43013311
:1061000013430B60FFF7EEF805230A689A43033B3D
:1061100013430B60FFF7E6F803232B70FFF7E2F859
:1061200060780B2866D84F4D494B03F06DF80C0092
:1061300014001C0024002D0036003E0046004E00D6
:1061400055005B004101A2781B689200A958CB184A
:10615000AB50FFF7C7F8A2781B689200A958CB1A7A
:10616000AB50FFF7BFF8A2781B689200A9584B43C9
:10617000AB50FFF7B7F8A4781968A400285903F0CA
:10618000D7F82851FFF7AEF8A4781968A400285969
:1061900003F0B4F92951FFF7A5F8A2781B68920023
:1061A000A9580B40AB50FFF79DF8A2781B689200EE
:1061B000A9580B43AB50FFF795F8A2781B689200E3
:1061C000A9584B40AB50FFF78DF81B68A278DB4312
:1061D0009200AB50FFF786F8A2781B689200AB5094
:1061E000FFF780F8A27818689200A958A8501960A3
:1061F000FFF778F803232B70FFF774F86078144EDC
:10620000174F0B2868D8A378164A9B0002F0F2FFBC
:106210000613172C32383C404447494DD358326856
:106220009B18336032680823002A58D13A68134318
:106230003B60FFF757F8D3583268D31AF1E7D358C9
:1062400032685343EDE7C04690F1FF1F10F2FF1F85
:106250003CF5FF1F50F5FF1F10F1FF1F42FAFF1F13
:10626000E4F4FF1F54F5FF1F3068D15803F060F8C5
:106270003060D7E7D158306803F040F93160D1E79A
:10628000D35832681340CCE7D35832681343C8E779
:10629000D35832685340C4E7D358DB43C1E7D358DF
:1062A000BFE73068D158D050E8E7D25833689A42F7
:1062B00006DA03233A689A43013313433B60B1E79C
:1062C0009A4204D106233A689A43053BF5E7052331
:1062D0003A689A43033BF0E703232B70A2E73A683E
:1062E0009A433A60FEF7FEFF60780B2865D8E34DCD
:1062F000E34B02F07FFF060E161E27303840484F52
:10630000555DA2781B689200A958CB18AB50FEF7D8
:10631000E9FFA2781B689200A958CB1AAB50FEF790
:10632000E1FFA2781B689200A9584B43AB50FEF7DF
:10633000D9FFA4781968A400285902F0F9FF285160
:10634000FEF7D0FFA4781968A400285903F0D6F806
:106350002951FEF7C7FFA2781B689200A9580B408D
:10636000AB50FEF7BFFFA2781B689200A9580B4301
:10637000AB50FEF7B7FFA2781B689200A9584B40BC
:10638000AB50FEF7AFFF1B68A278DB439200AB5027
:10639000FEF7A8FFA2781B689200AB50FEF7A2FFA1
:1063A000A27818689200A958A8501960FEF79AFFC1
:1063B000A2781B689200AA589AE603232B70FEF776
:1063C00091FFD3582A689B182B60FEF78BFFD35898
:1063D0002A68D31A2B60FEF785FFD3582A685343E7
:1063E0002B60FEF77FFF2868D15802F0A1FF2860DC
:1063F000FEF778FF2868D15803F080F82960FEF78F
:1064000071FFD3582A6813402B60FEF76BFFD358F7
:106410002A6813432B60FEF765FFD3582A68534060
:106420002B60FEF75FFFD358DB432B60FEF75AFF6C
:10643000D3582B60FEF756FFD15828682960D050FA
:10644000FEF750FFD2582B689A4200DA53E68D4986
:106450009A4200D058E606230A689A43053B134344
:106460000B60FEF73FFF03232B70FEF73BFF6078C6
:106470000B285ED802F0BEFE060E161E28323A42E7
:106480004A525D58A2787D4992005058C318535023
:10649000FEF728FFA278794992005058C31A53504A
:1064A000FEF720FFA278754992005058434353509D
:1064B000FEF718FFA478714DA4006059190002F08E
:1064C00037FF6051FEF70EFFA4786C4DA4006059B1
:1064D000190003F013F86151FEF704FFA278674931
:1064E0009200505803405350FEF7FCFEA2786349D7
:1064F0009200505803435350FEF7F4FEA2785F49D0
:106500009200505843405350FEF7ECFEA3785B498D
:106510009B005A58D2435A50FEF7E4FEA2785749DE
:1065200092005350FEF7DEFEA27854499200525872
:10653000DEE503232B70FEF7D5FEFCF7C9FA5249BE
:1065400001220B0040331A702279E37812021A43B9
:1065500063791B041A43A3791B0613434B64FEF7AC
:10656000C1FE6178454889000A58013A0A50002A5C
:1065700001DCFEF7B7FE444A5364FEF7B3FE434B1B
:106580001978E170597821719978DB786171A3717C
:10659000FDF742FAFEF7A6FE394B1B68FF2B01D927
:1065A000FEF7A0FE354A9B009958384B6960196088
:1065B0000822344B002904D119680A431A60FEF7F7
:1065C00091FE196891431960FEF78CFE2C4B1B68F5
:1065D000FF2B01D9FEF786FE2C4A9B001168274A43
:1065E0009950FEF77FFE2068000701D4FEF77AFE7F
:1065F000501C88649000264A1218486C4B64D06086
:10660000FEF770FE2068000701D5FEF76BFE501CF8
:10661000886490001E4A1218486C4B64D060FEF7E4
:1066200061FE2068C00701D4FEF75CFE501C886440
:106630009000174A1218486C4B64D060FEF752FE67
:106640002068C00701D5FEF74DFE501C88649000FD
:106650000F4A1218486C4B64D060FEF743FE206866
:10666000400701D4FEF73EFE501C88649000084AA3
:106670001218486C4B64D060FEF734FE54F5FF1FCF
:1066800050F5FF1FE4F4FF1F90F1FF1F3CF5FF1FC3
:1066900010F2FF1F05202468044201D1FEF722FEFC
:1066A000501C88649000384A1218486C4B64D060C3
:1066B000FEF718FE2068800701D4FEF713FE501C79
:1066C00088649000304A1218486C4B64D060FEF722
:1066D00009FE2068800701D1FEF704FE501C886483
:1066E0009000294A1218486C4B64D060FEF7FAFDFE
:1066F0002068C00601D4FEF7F5FD501C88649000A8
:10670000214A1218486C4B64D060FEF7EBFD2068FC
:10671000800601D4FEF7E6FD501C886490001A4AFA
:106720001218486C4B64D060FEF7DCFD2068400610
:1067300001D4FEF7D7FD501C88649000124A12184D
:10674000486C4B64D060FEF7CDFD2068000601D494
:10675000FEF7C8FD501C886490000B4A1218486C64
:106760004B64D060FEF7BEFD2068C00501D4FEF783
:10677000B9FD501C8864044892008218486C4B6430
:10678000D060FEF7AFFDC04610F2FF1FF0B5104C11
:1067900085B002AD8C462E002700019206CF06C6BA
:1067A00062460C4E190A72706A461279F370B27022
:1067B00000223171190C1B0EB371074B30701A7027
:1067C0007171FEF76DFB60680CCD0CC405B0F0BDB7
:1067D00048F5FF1FDCF4FF1F40F5FF1FF0B59D4D8E
:1067E0008BB02B005C331B789B4C002B03D19B4B55
:1067F0001B79002B0BD0FB22994B1B78991F114260
:1068000005D0EB3A93430F2B01D00023237022785D
:10681000531FD9B2012900D9A9E092488F49428A71
:1068200003925A1E934102AA073313704B79537097
:106830000023937062789A4200D08CE0838A02AA87
:106840001372894B02A81A7842725A788272DA79E6
:10685000C2729A7902735A7942731B7983738B7966
:10686000C37302A802F068FB002800D1A6E17F4BA9
:106870001B78002B25D07E4B7E4E1B78DAB2012A86
:1068800000D1C1E0002A18D0053B012B15D8754A6C
:1068900006A8938A31780372802343720A33837285
:1068A000817300230721C372037343730170437024
:1068B0008370538A436002F03FFB00236B4A3370BE
:1068C00013700023E27A237063709A4206D080210D
:1068D000694A5160694A1360FBF7E4FE02A802F0BE
:1068E000D3FA071E00D16BE102AA127A5C4B1A7030
:1068F00002AA527A5A7002AA927A9A7002AAD27A9C
:106900009A7102AA127B5A7102AA527B1A7102AAC8
:10691000927BDA7002AA514BD27B9A7102AA52780A
:106920005A71FBF7D7FD0022554B1860554B1A7072
:1069300002AB1B78072B00D08AE0023B23702B00B0
:1069400040331B785A1E012A00D89DE0052B00D148
:106950009AE0012299E0012A83D1A01C02A95A18C9
:10696000C118497801331172082BF7D179E7002358
:10697000012A3CD162789A422DD13A4F3A4E78782A
:106980003B783278C3189B1872789B18F2799B1861
:10699000B2799B1872799B1832799B18DBB20193FC
:1069A000FBF73EFE3878FBF73BFE3078FBF738FE0E
:1069B0007078FBF735FEF079FBF732FEB079FBF724
:1069C0002FFE7079FBF72CFE3079FBF729FE01983A
:1069D000FBF726FE4BE7012A00D048E71E00A31C68
:1069E000F05C0136FBF71CFE092EF8D13FE7022AC6
:1069F00000D03CE71C4E1B4F013A7370736032703D
:106A000078783B78C318C8E7164F327878783B78A7
:106A1000C3180A339B18DBB20193FBF701FE3878E9
:106A2000FBF7FEFD8020FBF7FBFD8A20FBF7F8FD5E
:106A30000020FBF7F5FD0020FBF7F2FD0020FBF73F
:106A4000EFFD3078FBF7ECFD0198FBF7E9FD34E74B
:106A5000062373E790F1FF1F10F2FF1F90F2FF1F54
:106A6000DCF4FF1F04F0FF1F48F5FF1F71FAFF1F42
:106A70003EFAFF1F73F9FF1F40F00F4000F0FF1FA9
:106A800034FAFF1F54F9FF1F00229E4B1A70290091
:106A900040310B78042B05D19B4E327853B2002B3A
:106AA00000DB04E102222378934301D0FEF7F8F9DA
:106AB0002378072B69D1FBF70DFDAA6E934E801A40
:106AC000C217336880185040984208D9904B1A7802
:106AD000012A01D101321A70FBF7FCFCA866FBF712
:106AE000F9FCEA6E7368801AC21780185040984209
:106AF00008D9874B5A78012A01D101325A70FBF725
:106B0000E9FCE866FBF7E6FC2A6FB368801AC21757
:106B100080185040984208D97D4B9A78012A01D1BB
:106B200001329A70FBF7D6FC28677A490B78002B64
:106B30002BD04B78002B28D1081D84461F00744AA7
:106B4000D05C022800D0A1E0664698008059461C1F
:106B500000D19AE0704A12686266704A1268A266B2
:106B60006A6C6864E2666E4A126822672A004C32D8
:106B700016786667266BA667E66AE66726006436BF
:106B800033770023137001334B702378072B06D122
:106B90002A0040321178022901D103311170A16B12
:106BA00000290BD0072B09D12B0040331B78012B78
:106BB00004D10023686C994200D96CE00BB0F0BDA1
:106BC00006A8FBF747FD002849D0FBF761FD554EAD
:106BD000002800D0F771F27902A9531C097CDBB2BE
:106BE000B218F3711172092B00D050E70023F37132
:106BF0004D4B327A1978914203D01979914200D0E5
:106C000045E71B799B1A59425941317131000023E4
:106C100008315A5C0133BF18FFB2082BF9D1337C1D
:106C2000BB4219D1384B727A1A70B27A5A70F27A22
:106C30009A70327B9A71727B5A71B27B1A71F27BB5
:106C4000DA70FBF747FC394B394A186000231370A0
:106C50000122F371227072E60223237017E72A00E3
:106C600040321378013B012B00D910E76B6C31499E
:106C70008B4208D85A1C180023496A6400F0A2F815
:106C80000723237065E6107001E7D75401332F2BDB
:106C900000D055E779E79A00A218D26B824203D15F
:106CA000052340352B7089E70133DBB283E70220EF
:106CB0002378834300D181E71F4DF3786A703279DE
:106CC000606B12021A4373791B041A43B3791B06D3
:106CD00013436B60174B98420ED8310000F092F9C5
:106CE0003100606B00F0F4F807230028DAD0636B02
:106CF000013363636523D5E707232B7000230B70F3
:106D00005CE7C04640F5FF1FDCF4FF1F18FAFF1FC9
:106D100042FAFF1F10F1FF1F3CF5FF1F50F5FF1F48
:106D2000E4F4FF1F90F2FF1F04F0FF1F38FAFF1F6B
:106D30003DFAFF1FFF07000048F5FF1F8023074AA9
:106D40001B0351690B4353615C22054B19780A43BD
:106D50001A7000225A7011329A70704700800440F5
:106D60000070074070B5002803D001281AD0002316
:106D700016E080242401114B20259C60104B1C0040
:106D8000DE782E42FCD05971E3785BB2002BFBDA3F
:106D90006379DBB2002A03D0002806D0012809D08D
:106DA000180070BD80242405E5E780210901034A0D
:106DB0005160F5E780210905F9E7C04600F00F4072
:106DC0000070074070B50724802344431B01E4187A
:106DD0000D00002203210120FFF7C4FF210AC9B2E0
:106DE00000220120FFF7BEFFE1B200220120FFF7E1
:106DF000B9FF002201201100FFF7B4FF0022287024
:106E000011000120FFF7AEFF002268701100012081
:106E1000FFF7A8FF0022A87011000120FFF7A2FFD2
:106E20000022E87011000120FFF79CFF002228716A
:106E300011000120FFF796FF012268710021100068
:106E4000FFF790FFA87170BD70B5802501242D015A
:106E5000220006212000FFF785FF002205212000E7
:106E6000FFF780FF002122002000FFF77BFF0221B7
:106E70000842F2D000222000FFF774FF290AC9B2AD
:106E800000222000FFF76EFFE9B200222000FFF78A
:106E900069FF002632003F3A53425A410021D2B2E4
:106EA00020000136FFF75EFF402EF3D100220521BE
:106EB0002000FFF757FF220000212000FFF752FFBC
:106EC0002042F3D180234035DB019D42C0D170BD0B
:106ED000F7B50724802344431B01E4180D0000226A
:106EE00003210120FFF73EFF210AC9B20022012041
:106EF000FFF738FFE1B200220120FFF733FF002245
:106F000001201100FFF72EFF0022070011000120D1
:106F1000FFF728FF0022060011000120FFF722FFE3
:106F20000022040011000120FFF71CFF6B46002225
:106F3000D87011000120FFF715FF6B460022187171
:106F400011000120FFF70EFF6B460122587100214E
:106F50001000FFF707FF6B4698712B780020BB42AB
:106F600017D16B78B34214D1AB78A34211D16B46E1
:106F70000198DB7800022A790343E8781202024381
:106F8000687900040243A87900061043181A4342A6
:106F90005841FEBD012270B504000D00100006210D
:106FA000FFF7E0FE0126002205213000FFF7DAFEA0
:106FB000002132003000FFF7D5FE02210842F2D056
:106FC00000220120FFF7CEFE210AC9B200220120D3
:106FD000FFF7C8FEE1B200220120FFF7C3FE012245
:106FE00029001000FFF7BEFE012400220521200029
:106FF000FFF7B8FE220000212000FFF7B3FE204279
:10700000F3D170BD70B5072480230D0044431B01EC
:10701000E0180978FFF7BEFF0F4B6978E018FFF71B
:10702000B9FF0E4BA978E018FFF7B4FF0C4BE978D5
:10703000E018FFF7AFFF0B4B2979E018FFF7AAFF25
:10704000094B6979E018FFF7A5FF084BA979E0180B
:10705000FFF7A0FF70BDC046010800000208000055
:1070600003080000040800000508000006080000EE
:10707000F7B5170001220191050006211000FFF766
:1070800071FE0124002205212000FFF76BFE002184
:1070900022002000FFF766FE02210842F2D0002203
:1070A0000120FFF75FFE290AC9B200220120FFF785
:1070B00059FEE9B200220120FFF754FE0026012408
:1070C000BE420DD10124002205212000FFF74AFE17
:1070D000220000212000FFF745FE2042F3D1F7BD3A
:1070E000019B0135995D3F232B4000932200002B2B
:1070F00004D07A1E921B53425A41D2B22000FFF7AD
:1071000031FE009B002B2FD17B1E9E422CD20022F1
:1071100005212000FFF726FE220000212000FFF7B6
:1071200021FE2042F3D1220006212000FFF71AFEA3
:10713000002205212000FFF715FE0021220020007B
:10714000FFF710FE02210842F2D000222000FFF7D4
:1071500009FE290AC9B200222000FFF703FEE9B2A6
:1071600000222000FFF7FEFD0136A9E710B504005C
:10717000002203210120FFF7F5FD210AC9B20022F8
:107180000120FFF7EFFDE1B200220120FFF7EAFD49
:10719000012200211000FFF7E5FD10BD70B50400CD
:1071A0000E001500032100220120FFF7DBFD210A5C
:1071B000C9B200220120FFF7D5FDE1B20022012073
:1071C000FFF7D0FD0024AC4200D170BD6A1E121B37
:1071D00053425A410021D2B20120FFF7C3FD30557E
:1071E0000134F0E773B56B469C1D022221001B4859
:1071F000FFF7D4FF22881A4B1A4D9A4203D11A4B3B
:107200001B78002B19D0002602222100134826806B
:10721000FFF72EFFFFF718FE202229003000FFF7AE
:1072200027FF402211491000FFF722FF104B0222D6
:1072300021000A482380FFF71BFF2900202200209D
:10724000FFF7ACFF40220B491000FFF7A7FF4C22CD
:1072500009490A4804F064FB73BDC046FE070000FC
:10726000A5A5000004F0FF1F80F9FF1FE0BE00008D
:10727000A5A5FFFF84F9FF1F94BE0000C8F9FF1FFA
:10728000034B185C053843425841C0B27047C046B2
:10729000A4F2FF1FF0B5B84B85B019698022B74B37
:1072A000B74C89002FD59A600022A378E318E578BF
:1072B0005A70002D09D1E8B2FBF78EFA231DE8546D
:1072C0000135082DF7D10123E37000250226E8B22D
:1072D000FBF782FA231DEA5C824229D0E854A94BCD
:1072E0005B199B7CDBB2022B19D0032B03D0012B43
:1072F0001ED100281CD02B00A34A2733D15C0129C2
:1073000016D1D65414E05A60A07823185B78002B6D
:1073100001D100F016FCA3780122E318C7E700288A
:1073200006D12A0098492732885C012800D18B5465
:107330000135082DCBD1954DAB68002B13D0944F60
:107340003E78002E0FD1FBF7C5F8924B1B68C01A90
:10735000C317C0185840AB68984204D901233000C5
:107360003B7000F0EEFB2B8B002B13D08A4F3E7846
:10737000002E0FD1FBF7AEF8884B1B68C01AC3175D
:10738000C01858402B8B984204DD012330003B701D
:1073900000F0D7FB2221A07800F044FB0600A07883
:1073A00000F0B8FB0F210500A07800F03BFB442360
:1073B0000390A0787A4F4343FB181B69002B27D01A
:1073C0003602F217B6185640DA179B1853409E4201
:1073D0001EDD23181B7B002B08D180220121D20443
:1073E00000F05EFB0122A378E3181A7300230293D6
:1073F000EB071DD5A078644AC31CD15C012914D1C8
:107400000131D154012100F091FB012302930FE0DF
:1074100023181B7B002BE9D080220121D20400F02D
:107420004CFBA3780022E318DFE7D35C002BE9D004
:10743000AB0010D5A078544A03000F33D15C01296A
:1074400001D10131D1548021890500F06FFB012168
:10745000A378544AD1542900534B1940994202D180
:10746000A07800F063FB2900504B1940994202D1EB
:10747000A07800F05BFB29004D4B1940994202D1E6
:10748000A07800F053FB29004A4B1940994202D1E1
:10749000A07800F04BFB4423A0784343FB185B6AC1
:1074A000002B22D08026F60235421ED000F049FB88
:1074B0005021A07800F0B6FA0200A0783E4B81007F
:1074C000CB582121D21A00F089FA3100A07800F0BF
:1074D0002DFBA1782C4A0B001533D05C012801D17B
:1074E0000130D0540122354B5A548022039B1A405C
:1074F000A378002A13D0E218517B002920D1013152
:107500005173204AD218127C0A4219D08B401E4A6D
:107510001B33D15C012913D10131D15410E0E118A2
:10752000487B00280CD04A730221164AD218127CDC
:107530000A4205D05B00144A1B33D05C0128ECD012
:107540008022039B520013401A00A378002A37D0F0
:10755000E218917B002944D101319173094AD21874
:10756000527C0A423DD00E338B40074AD15C012940
:1075700037D10131D15434E000F00F4040F00F40DA
:10758000A4F2FF1F18FAFF1F42FAFF1F04F0FF1FAB
:107590003DFAFF1F38FAFF1F54F9FF1F34FAFF1F8F
:1075A00084F9FF1F81F9FF1F080800000810000080
:1075B000082000000840000074F9FF1F71F9FF1F48
:1075C000E118887B00280CD08A730221AC4AD218BB
:1075D000527C0A4205D00E33AA4A5B00D05C0128D7
:1075E000C8D002210D4211D0A078A64A0300093369
:1075F000D55C012D04D1D154022100F097FA05E0A9
:10760000D35C002BF8D0029B002BF5D1FAF762FF78
:107610002369C01AC317C01858400A2839DDA0785A
:10762000994D9A4B9A4A8100C3188218491901F062
:1076300051FBA578605D052823D801F0DBFD032C04
:10764000748C9ED74C236B43924A9B5C002B18D0C2
:10765000280000F0CBFE002813D11021280001F0F3
:1076600007F844226A438C4B10219B185A7A8B4BA3
:10767000D208184012020243280000F0CBFF012379
:107680006355A07800F094FB0023A370FAF722FF63
:10769000206105B0F0BD00220521280000F09EF910
:1076A0004C236B437B4A2800D218117D937D0191B6
:1076B000527D06210092002200F068F9792128000D
:1076C00000F0B0F980267F2805DD8023FF33984243
:1076D0001CDCC0267600361A04222021280000F087
:1076E0007DF96F4A2421280000F078F92121280033
:1076F00000F098F937218219280000F06FF9FAF7A5
:10770000E9FEAB00E31858610223B9E7654BA026F8
:10771000984203DD644B984202DCE026B600DAE7CB
:107720009026F600D7E7FAF7D5FEAB00E3185B69C1
:10773000C01AC317C0185840FA239B009842A0DD16
:107740002121280000F06EF950210200280000F0ED
:1077500045F9032394E7C02207215205280000F0D1
:10776000ACF9524A0721280000F09AF9FAF7B2FE64
:10777000AB00E3185861042382E7FAF7ABFEAE00D2
:10778000A3195B69C01AC317C0185840FA239B009D
:10779000984200DC75E7992207211206280000F0C4
:1077A0008CF9A02207211205280000F079F9802227
:1077B0000521280000F012F95921280000F032F9C3
:1077C0004C226A43334B50219B1800221861384BDE
:1077D0002800F25000F026F921210700280000F0CF
:1077E00021F9344B381AF050052349E74C236B43F9
:1077F000284A9E5C002E00D043E780220721D20356
:10780000280000F05AF903220521280000F0E6F8CC
:1078100044236B43FF18BB7DBA7A01937B7A062120
:1078200000932800330000F0B1F81021280000F088
:107830001FFFF822520102431021280000F0EAFE47
:10784000FB7D66550122002B00D00222202128005A
:1078500000F0C4F800222421280000F0BFF8212104
:10786000280000F0DFF8124BAA00D2582121821A1A
:10787000280000F0B3F801220F4B5A5501E7C0462B
:1078800018FAFF1F42FAFF1F7CF9FF1F82F9FF1F42
:1078900064F9FF1FC8F9FF1F84F9FF1FFFE0FFFF16
:1078A00040420F007F0200007F0300000000408183
:1078B00060F9FF1F74F9FF1F72F9FF1F704710B5C1
:1078C000FAF708FE054C2368C01AFA235B009842B9
:1078D00002D9FAF7FFFD206010BDC04674FAFF1F01
:1078E00010B5244B5A78012A1FD0002A05D0022A4D
:1078F0002DD00322204B1A7010E01979DA78090292
:1079000011435A799878120411439A7912060A435E
:1079100005D180229204072100F0CFF810BD80220B
:107920009204072100F0BCF8F8E71979DA78090227
:1079300011435A799878120411439A7912060A432E
:1079400002D180221205E6E780221205E9E71979C3
:10795000DA78090211435A799878120411439A7916
:1079600012060A4302D180225205D4E78022520532
:10797000D7E7C046DCF4FF1F48F5FF1F704770478C
:1079800070477047704770477047C046F7B51E0094
:1079900008AB1D7809AB1B78170001930E4B002232
:1079A0001C5C802320001943FFF7DCF9390000221A
:1079B0002000FFF7D7F9310000222000FFF7D2F9AD
:1079C000290000222000FFF7CDF9012201992000B3
:1079D000FFF7C8F9F7BDC046BCF2FF1F70B5104BEA
:1079E00014001D5C8023280019430022FFF7BAF918
:1079F000210E28000022FFF7B5F921142800C9B292
:107A00000022FFF7AFF921122800C9B20022FFF7C8
:107A1000A9F92800E1B20122FFF7A4F970BDC04620
:107A2000BCF2FF1F70B51D4B00221C5C0D00200036
:107A3000FFF798F9002220001100FFF793F90022C8
:107A400020001100FFF78EF9002220001100FFF73F
:107A500089F9012200212000FFF784F92900002282
:107A60002000FFF77FF9002220001100FFF77AF9CC
:107A70000022060211002000FFF774F900223043B3
:107A8000110005022000FFF76DF9012205430021D6
:107A90002000FFF767F92D02284370BDBCF2FF1FDD
:107AA00070B516000D000400FFF7BCFF02002900AE
:107AB00032432000FFF792FF70BD70B516000D0035
:107AC0000400FFF7AFFF02002900B2432000FFF7D8
:107AD00085FF70BDF7B51C0008AB1D780F00009244
:107AE0000600FFF79FFF29190191220000230121C1
:107AF000019DAA4209D3009A3900A24042401A408F
:107B000042403000FFF76AFFF7BD0D00954001329B
:107B10002B43EDE7012210B5040052420C21FFF780
:107B20005DFF0E212000FFF77DFF10BD10B50400A2
:107B3000CA430C21FFF752FF0E212000FFF772FF0E
:107B400010BD10B5040000222021FFF747FF0022DE
:107B500024212000FFF742FF10BD37B5002180220D
:107B6000002408005201FFF739FF6C4A1021002061
:107B7000FFF734FF6A4A04210020FFF72FFF694A0C
:107B80000C210020FFF72AFF0E210020FFF74AFFFB
:107B900023000194009422006D212000FFF7F6FEDF
:107BA00022006C212000FFF719FF0322052120008D
:107BB000FFF714FF042220212000FFF70FFF22000F
:107BC00037212000FFF70AFF220021212000FFF7C4
:107BD00005FFC825C822AD02120424212000FFF7AA
:107BE000FDFE2A0028212000FFF7F8FE2A002921A7
:107BF0002000FFF7F3FE4C4D0621AB7DAA7A0193DE
:107C00006B7A200000932300FFF7C0FEAB8A474A3F
:107C100015215A432000FFF7E1FE454D60216A68B7
:107C20002000FFF7DBFEAA6861212000FFF7D6FEE7
:107C30002A7BEB8912041A431C212000FFF7CEFE99
:107C40002A6959212000FFF7C9FE2A6A5A2120001B
:107C5000FFF7C4FE6A6A5B212000FFF7BFFE2822FF
:107C60002C23AA181278EB181B780192AA6A5D21BE
:107C7000120AD2B2009220002200FFF787FE2A6B80
:107C80005E212000FFF7AAFEAA6918212000FFF755
:107C9000A5FEEA6919212000FFF7A0FE6A6B5C21AE
:107CA0002000FFF79BFEAA6B5F212000FFF796FEE6
:107CB000EA6B52212000FFF791FE29004423403156
:107CC0000978EB186A6C1B78019129004131097819
:107CD000120A00914835D2B263212000FFF756FE08
:107CE0002B782200019400947D212000FFF74EFEA6
:107CF00002212000FFF71AFF02220D212000FFF7CA
:107D0000CFFEC022012192022000FFF767FE094A40
:107D100035212000FFF762FE37BDC0460500050093
:107D20008D123083FFFFFFFD84F9FF1F00710200F9
:107D3000C8F9FF1FFFFFFF7F10B521210400FFF7E7
:107D400071FE064B3521C2182000FFF747FE0F21B8
:107D50002000FFF767FEC004C00F10BDFFFFFF7FCC
:107D60000002704780007047001270478010704713
:107D70007047C046442242430C4B70B59B18DB7DD4
:107D800004000D000122002B00D00222200020213F
:107D9000FFF724FE8022200052050721FFF780FE16
:107DA0002A0024212000FFF719FE70BD84F9FF1F6F
:107DB000F0B50F2185B00400FFF734FE4422624382
:107DC000D04B012599180B7A49685E0643D5070AFE
:107DD000C00928400390CB482F40125852420292CB
:107DE0004A4201923F251D405BB20020002B3CDA45
:107DF000FFF7A2FF43424341DBB20A2D00D9CFE196
:107E00000122C021AA40C9000A4200D06CE2F02140
:107E100049000A4200D04AE11E231A4200D1BFE1C4
:107E2000B94E305D0138122800D9B9E101F0ECF902
:107E30002300320041004F005E00660075008300A1
:107E4000C100F500FA00B8013701B801B801B80166
:107E5000B80153029A02C709000A28400390A948B2
:107E60002F40125801910292BCE7FFF765FF431EB5
:107E70009841C3B2C1E701212000FFF7D3FD0122E1
:107E8000A300F3185860A14B023D1A5595421BD828
:107E900002231AE0A300F3185B6802221A430121AF
:107EA0002000FFF79BFD02992000FFF763FF0323EB
:107EB0000BE0039B002B00D172E121212000FFF792
:107EC000B1FD934BA200D0500423335568E1A300C9
:107ED000F3185A6801210A432000FFF77FFD029B37
:107EE00020005942FFF746FF0523EEE7002F00D19F
:107EF00056E12000FFF725FE0623E6E7A300F3186E
:107F00005A680323012120009A43FFF767FD019976
:107F10002000FFF72FFF0723D7E7002F00D03FE116
:107F200039002000FFF726FF019B20005942FFF790
:107F300021FF0823C9E7002F00D131E121212000D2
:107F4000FFF770FD050000212000FFF713FF7049C7
:107F5000A3005A582000521B5A50F3185A680323A2
:107F600001219A43FFF73AFD44236343654AD3183E
:107F7000DB7D0522002B00D0062220212000FFF708
:107F80002DFD019A24212000FFF728FD80220721E2
:107F900052052000FFF791FD8022072112052000E5
:107FA000FFF77EFD2A0037212000FFF717FD092388
:107FB0008BE70F212000FFF735FDC30700D4EFE06A
:107FC00021212000FFF72EFD524B002118602000D8
:107FD000FFF7D0FE4C2363434F4A9F5C002F09D12B
:107FE0003A0037212000FFF7F9FC3A002121200058
:107FF000FFF7F4FC21212000FFF714FD474BA700F9
:10800000F85050212000FFF70DFD454B033DF8507F
:10801000012D4AD8019B5942D6E0002F00D1BFE084
:108020000B2352E7002F00D0BAE021212000FFF7F8
:10803000F9FC050039002000FFF79CFEEB0F5D19ED
:10804000A300F3185A68032301219A432000FFF785
:10805000C5FC442363432B4A6D10D318DB7D0522F6
:10806000002B00D0062220212000FFF7B7FC019A48
:1080700024212000FFF7B2FC8022072152052000B6
:10808000FFF71BFD8022072112052000FFF708FDE6
:108090002A0037212000FFF7A1FC0D2315E70F214F
:1080A0002000FFF7BFFCC3077AD512230DE7164E59
:1080B000305D0138122873D801F0A6F8130034009F
:1080C00046005500670072007400720072009C0048
:1080D000A6008B00DC0072007200720072000D01BD
:1080E00054010121094B20001955FFF79BFCA30007
:1080F000F31858600223063D9D43EDB2002D00D0D9
:10810000E2E6E2E684F9FF1FC0F2FF1F72F9FF1FEB
:1081100058F9FF1F14FAFF1FC8F9FF1F60F9FF1F6E
:1081200074F9FF1F062D06D1A300F3185A68032324
:108130009A431300B1E6082D00D0B4E6A300F3186B
:108140005A6803239A43AAE66A1F012A07D8039AAA
:10815000002A04D0062D00D1B6E61323B5E6002B85
:108160001ED00C23B1E6052D05D1A300F3185A68E3
:1081700003239A43AEE6072D00D0B0E6A300F31820
:108180005A68032301219A43A6E66A1F012A04D8EC
:10819000002F02D0052DE0D17AE6002B00D0BAE600
:1081A00005B0F0BD002BFBD1073D012D0BD9A3007D
:1081B000F3185A6803239A431300022201211A4339
:1081C0002000FFF70BFC01992000FFF7D3FD0A23E5
:1081D0007BE6002BE4D1073D012D00D81AE7A30070
:1081E000F3185A68032301219A430A432000FFF73A
:1081F000F5FB0FE7002BD3D021212000FFF712FC65
:10820000A300F31898600BE7002BC9D121212000AF
:10821000A500FFF707FC73195A68032302909A43DD
:1082200001212000FFF7DAFB442363435D4AD318A2
:10823000DB7D0522002B00D0062220212000FFF745
:10824000CDFB019A24212000FFF7C8FB80220721E3
:1082500052052000FFF731FC802277191205072113
:108260002000FFF71DFCBA68029B9D18EA0F521907
:1082700052100EE70F212000FFF7D4FBC30700D4F4
:108280008EE71223212120003355FFF7CBFB464B0D
:10829000002118602000FFF76DFD4C236343434A23
:1082A0009D5C002D09D12A0037212000FFF796FBA5
:1082B0002A0021212000FFF791FB21212000FFF758
:1082C000B1FB3B4BA500E85050212000FFF7AAFB73
:1082D000384BE85064E7A300F3185A6801212000E6
:1082E000FFF77CFB0023F0E5334E335D0D2B4ED0C2
:1082F00033D8012B3BD00A2B00D051E70E212000B0
:10830000FFF790FBC30300D44AE700212000FFF7EA
:1083100031FD44236343234AD318DB7D0522002B20
:1083200000D0062220212000FFF758FB019A2421CB
:108330002000FFF753FB8022072152052000FFF7A2
:10834000BCFB8022072112052000FFF7A9FB362184
:108350002000FFF767FB02009BE6122BC2D0132B15
:1083600000D01DE700212000FFF704FD9DE69021CD
:10837000124A090320001355FFF7D8FB104A0721C2
:108380002000FFF78DFB092D00D043E61BE70F21EE
:108390002000FFF747FB0123184200D100E711330B
:1083A00070E7C04684F9FF1F14FAFF1FC8F9FF1FCA
:1083B00060F9FF1F74F9FF1FC0F2FF1F72F9FF1F62
:1083C000680A0000034B1A5C002A01D101321A54DA
:1083D0007047C046C0F2FF1F034B1A5C002A01D051
:1083E00013221A547047C046C0F2FF1F014B185C9D
:1083F0007047C046C0F2FF1F0C2313B51D4C0A2165
:10840000228C00200093083BFFF764FB00218022B0
:1084100008005201FFF7E2FAE3690020D9175A1861
:108420004A405421FFF7DAFA8022E36992050721D6
:108430000020002B1ADAFFF733FB00225021100036
:10844000FFF7CCFA0C4BFF201A00403210701A00D4
:108450000821413211705A6C0190D3B2CA40009188
:10846000D2B25B310020FFF791FA13BDFFF725FB75
:10847000E3E7C04684F9FF1FC8F9FF1F70B50C0081
:1084800007210500FFF7CEFA802302009A43E10797
:1084900001D503431A00A3073BD580235B001A4391
:1084A000102113008B43600701D50B0013432207F3
:1084B00032D580229200134304211A008A43E00639
:1084C00001D50A001A43082113008B43A00601D5E9
:1084D0000B00134320211A008A43600601D50A00CD
:1084E0001A43402113008B43200601D50B00134390
:1084F00002211A008A43E00501D50A001A43A305A8
:108500000DD58023DB001A4328000721FFF766FA08
:1085100070BD044B1A40C3E7034A1340CCE7034B3A
:108520001A40F1E7FFFEFFFFFFFDFFFFFFFBFFFF2C
:1085300010B50721FFF776FA03000006C00FDA0531
:1085400001D502221043DA0601D5042210439A0510
:1085500001D5082210435A0701D5102210432021CB
:108560001A0700D5084340220B4200D010431342A3
:1085700001D0802210439A0702D580225200104376
:108580005B0502D580239B00184310BDF0B50400A5
:1085900085B01D000AAB1B780291160003931B4A9D
:1085A0000BAB0C211F78FFF719FA0E212000FFF703
:1085B00039FA8023029A6D2113430022019300921D
:1085C00013002000FFF7E2F9039B019700933200AC
:1085D0002B006C212000FFF7D9F90E212000FFF7B6
:1085E00021FA80239B041842F7D036023543039BBF
:1085F0002D022B431D027F23029A3D431A4014197A
:10860000034BA400E55005B0F0BDC046FFFFFFFDE1
:10861000CCF2FF1FF7B506000C0015000C21124A22
:10862000FFF7DCF90E213000FFF7FCF98023002270
:1086300023430193009213006D213000FFF7A6F948
:1086400080272A006C213000FFF7C8F9BF040E21F3
:108650003000FFF7E7F93842F9D07F231C40A41916
:10866000024BA400E550F7BDFFFFFFFDCCF2FF1F5A
:1086700073B57F241B4B0C401B5D0500002B2BD0DA
:108680000026194A0C21FFF7A9F90E212800FFF74F
:10869000C9F93300320000966D2128000194FFF7DC
:1086A00075F932006C2128008026FFF797F9B6048F
:1086B0000E212800FFF7B6F93042F9D06E212800CC
:1086C000FFF7B0F9DF23223C1C4204D1030202D59C
:1086D000FF231B06184376BD2418044BA400E05862
:1086E000F9E7C04624BF0000FFFFFFFDCCF2FF1FEB
:1086F00070B50D006C210400FFF7BAFF02000F20D7
:10870000054082432A436C212000FFF783FF70BDA0
:1087100070B50C006C210500FFF7AAFF7023220141
:1087200098431A4002436C212800FFF773FF70BD85
:1087300070B50C006C210500FFF79AFFE203C0241E
:1087400064022240034C6C21204002432800FFF7C2
:1087500061FF70BDFF7FFEFF70B50C006C2105004E
:10876000FFF786FF2205F02424042240034C6C21ED
:10877000204002432800FFF74DFF70BDFFFF0FFFB1
:1087800070B50C006C210500FFF772FF2206F02483
:1087900024052240034C6C21204002432800FFF7AF
:1087A00039FF70BDFFFFFFF070B50D006C210400B4
:1087B000FFF75EFF002D07D08022D20502436C2117
:1087C0002000FFF727FF70BD014A0240F7E7C046CF
:1087D000FFFFFFBF70B50D006C210400FFF748FFDD
:1087E000002D07D08022120302436C212000FFF7E6
:1087F00011FF70BD014A0240F7E7C046FFFFF7FFD7
:1088000070B50D006C210400FFF732FF002D07D07A
:108810008022D20202436C212000FFF7FBFE70BDD4
:10882000014A0240F7E7C046FFFFFBFF70B50D00AD
:108830006C210400FFF71CFF002D07D08022D2011D
:1088400002436C212000FFF7E5FE70BD014A0240A3
:10885000F7E7C046FFBFFFFF70B50D006C210400B5
:10886000FFF706FF002D07D08022920102436C2102
:108870002000FFF7CFFE70BD014A0240F7E7C04677
:10888000FFDFFFFF70B50D006C210400FFF7F0FE65
:10889000002D07D08022520102436C212000FFF7F7
:1088A000B9FE70BD014A0240F7E7C046FFEFFFFF87
:1088B00070B50C006C210500FFF7DAFE23070DD51B
:1088C0007023802298431201104322017024224019
:1088D00002436C212800FFF79DFE70BD014A104045
:1088E000F3E7C0468FF7FFFF70B50C006C21050061
:1088F000FFF7BEFEE201F024E4002240034C6C21AD
:10890000204002432800FFF785FE70BD7FF8FFFF7F
:1089100010B5FFF7E9FF10BD70B50D006C21040024
:10892000FFF7A6FE002D07D08022920202436C21A1
:108930002000FFF76FFE70BD014A0240F7E7C04616
:10894000FFFFFDFF10B56C21FFF792FE0F231840CB
:1089500010BD10B56C21FFF78BFE4006400F10BD17
:1089600010B56C21FFF784FEC003800F10BD10B559
:108970006C21FFF77DFE0002000F10BD10B56C21C9
:10898000FFF776FE0001000F10BD10B56C21FFF758
:108990006FFE4000C00F10BD10B56C21FFF768FEE0
:1089A0000003C00F10BD10B56C21FFF761FE40033E
:1089B000C00F10BD10B56C21FFF75AFE4004C00F68
:1089C00010BD10B56C21FFF753FE8004C00F10BD21
:1089D00010B56C21FFF74CFEC004C00F10BD10B5E0
:1089E0006C21FFF745FE02004006400F130501D53C
:1089F0000823184310BD10B56C21FFF739FE400560
:108A0000000F10BD10B5FFF7F6FF10BD10B56C21BB
:108A1000FFF72EFE8003C00F10BD70B50C006D2156
:108A20000500FFF725FE6023620198431A400243C8
:108A30006D212800FFF7EEFD70BD70B50C006D21B3
:108A40000500FFF715FE6203C024E4012240044C38
:108A50006D21204002432800FFF7DCFD70BDC046B9
:108A6000FF9FFFFF70B50C006D210500FFF700FEB2
:108A70002202F02424012240034C6D2120400243B5
:108A80002800FFF7C7FD70BDFFF0FFFF70B50D00B8
:108A90006D210400FFF7ECFD02000F20054082432A
:108AA0002A436D212000FFF7B5FD70BD70B50D00A4
:108AB0006D210400FFF7DCFD044A2D0402402A4327
:108AC0006D212000FFF7A6FD70BDC046FFFF00FF2F
:108AD00070B50D006D210400FFF7CAFD002D07D011
:108AE0008022120202436D212000FFF793FD70BD2A
:108AF000014A0240F7E7C046FF7FFFFF70B50D0057
:108B00006D210400FFF7B4FD002D07D08022520430
:108B100002436D212000FFF77DFD70BD014A024038
:108B2000F7E7C046FFFFFFFE10B56D21FFF7A0FD80
:108B30004006800F10BD10B56D21FFF799FD400470
:108B4000800F10BD10B56D21FFF792FD0005000FDD
:108B500010BD10B56D21FFF78BFD0F23184010BD20
:108B600010B56D21FFF784FD0314D8B21B0601D5A3
:108B7000014B184310BDC04600FFFFFF10B56D212B
:108B8000FFF776FD0004C00F10BD10B56D21FFF793
:108B90006FFDC001C00F10BD70B50C007021050045
:108BA000FFF766FD054A702110400322224012059E
:108BB00002432800FFF72EFD70BDC046FFFFCFFF28
:108BC00070B50D0070210400FFF752FD002D07D095
:108BD00080221203024370212000FFF71BFD70BDAD
:108BE000014A0240F7E7C046FFFFF7FF70B50D00EE
:108BF00070210400FFF73CFD002D07D08022D20237
:108C0000024370212000FFF705FD70BD014A0240BC
:108C1000F7E7C046FFFFFBFF70B50C0070210500B1
:108C2000FFF726FD054A702110400322224012045E
:108C300002432800FFF7EEFC70BDC046FFFFFCFFBB
:108C400070B50C0070210500FFF712FD044A2402E4
:108C50000240224328007021FFF7DCFC70BDC046B3
:108C6000FF00FFFF70B50C0070210500FFF700FD4D
:108C7000FF2302009A43280022437021FFF7CAFC19
:108C800070BD10B57021FFF7F3FC8002800F10BD9E
:108C900010B57021FFF7ECFC0003C00F10BD10B53C
:108CA0007021FFF7E5FC4003C00F10BD10B5702127
:108CB000FFF7DEFC8003800F10BD10B57021FFF7B9
:108CC000D7FC000AC0B210BD10B57021FFF7D0FC70
:108CD000C0B210BD70B50E006C2115001C00FEF76F
:108CE000A1FE002E02D083059B0D3360002D02D023
:108CF000C302DB0E2B70002C01D0000E207070BD63
:108D000013B5F9F7E7FB0400F9F7E4FB001BC31701
:108D1000C01858400928F7DD00211B4A0800FFF75A
:108D200079FC532300220193513B009310003F3301
:108D30006C21FFF72BFC06230193033B00930023D8
:108D400009211A0018000024FFF720FC0A21220044
:108D50000191200000940123FFF718FC1F2322003B
:108D600001930093200023001021FFF70FFC074A16
:108D700070212000FFF74EFC2000FFF7E3FD044BBD
:108D800018705C7013BDC046010001001E000CC4C9
:108D9000CCF4FF1FF8B5064D04002E187178002999
:108DA00005D12F5CFFF7A4FC01232F557370F8BD8C
:108DB000CCF4FF1F10B5054B1A185178002904D0C8
:108DC00000215170195CFFF793FC10BDCCF4FF1F1C
:108DD000802330B52A4C1B0265692B436361012453
:108DE000284B1D7825431D705D782542FCD0032556
:108DF0005C7802382C407D352C435C7006283AD8CC
:108E00001C2400F0F7F9363432302E2C0400802078
:108E10009870DC700020CC08E4B2D8721C7407246F
:108E20004901C9B259749874D87418755C759875ED
:108E3000D87582420BD0D1085201C9B2D2B219768C
:108E40005A769876D87618775C779877D877012213
:108E500019789143197059781142FCD130BD8120A5
:108E6000D6E78320D4E78720D2E78920D0E7932074
:108E7000CEE7B120CCE7832098706738D870C9E777
:108E80000080044000400240F7B50124234902005D
:108E90000B7900200191234234D008252048C37F5C
:108EA0002B40204D2FD05470EB7F1F4DC67FC07FCD
:108EB000ED7F5B05AC466146C9010B4380211B4D2C
:108EC00009060B43E021EF7FC003E7408902084019
:108ED000034370093B43800403435360EB7F23400B
:108EE0009370002312495818C47FD01801330472BC
:108EF000082BF7D10F200F4B1B7803401370019BF9
:108F00000E381871FEBD5370EB7FC57FDB006D0915
:108F10002B435360C37F1B09E1E7C046004002407A
:108F2000024002400140024003400240044002402F
:108F3000054002402C400240F0B501272B4C0500B3
:108F4000A37900203B423CD0A7726A682848294B8D
:108F5000002A37DA510DC9B2017018201978960C21
:108F600001401038014376010E439103490F0E432F
:108F7000F6B21E70D109204EC9B231701F4E317841
:108F8000394057003943C9B2317019780843187015
:108F900000216818067A1A48081801310670082955
:108FA000F7D10F2617482D780178B1432943017076
:108FB000002A16DA0121114A13788B43137001201D
:108FC000A071F0BDD108C9B2017017201978014015
:108FD000500101430820C9B21970197881431970F2
:108FE000D6E710211A788A431A70E8E70040024059
:108FF00030400240314002403240024033400240A3
:10900000344002403C4002401FB500236A46937042
:10901000537008331370073B01931372223353725A
:10902000223393722233D372223313732233537356
:109030002233937368462233D373FFF77DFF05B065
:1090400000BDC04600BE704710B5044B044A9A608C
:1090500000F05AF800F08CF810BDC04600ED00E0BA
:1090600000200000202801DDC0467047074B184053
:1090700004D5202301385B42184301300123C0216D
:109080008340034A490053501360EEE71F000080FD
:1090900000E100E0202801DDC0467047064B184083
:1090A00004D5202301385B4218430130012383405B
:1090B000024AD367F1E7C0461F00008004E100E0E8
:1090C00010B503291BDC202819DC0322C317134029
:1090D0001B18FC329B1089011340094C1140094AAE
:1090E0009B001B19104004D5042201385242104342
:1090F0000130C0B2C00081401A681143196010BD30
:1091000000E400E003000080144B154A0F219A8010
:1091100001225A7022321A700022124B5A62124BEC
:109120005A780A405A70114A853111709A221A7081
:109130008A3A19791142FCD10C211A790A40082A7D
:10914000FBD10F215A78114010220A430C215A708A
:109150001A790A40082AFBD17047C0460020054012
:1091600003E8FFFF00800440004006400050064036
:109170003F2270B51A4C2378934323D104252378DA
:109180002B421CD10121237816489B065B0F994086
:1091900000F044F8144B1B782B4200D04009A02368
:1091A000DB005843114A6378516A5B098900890FD3
:1091B000D840013100F032F80D4B186070BD8020AE
:1091C0000002ECE723789343402B05D023789343A8
:1091D000802BF3D10348E5E780200002E2E7C04698
:1091E000004006400024F400005006400080044087
:1091F00024F0FF1F02B4714649084900095C490088
:109200008E4402BC7047C04603B471464908400012
:109210004900095A49008E4403BC704700224308A4
:109220008B4274D303098B425FD3030A8B4244D32E
:10923000030B8B4228D3030C8B420DD3FF22090270
:1092400012BA030C8B4202D31212090265D0030B2F
:109250008B4219D300E0090AC30B8B4201D3CB0325
:10926000C01A5241830B8B4201D38B03C01A524167
:10927000430B8B4201D34B03C01A5241030B8B4269
:1092800001D30B03C01A5241C30A8B4201D3CB0254
:10929000C01A5241830A8B4201D38B02C01A524139
:1092A000430A8B4201D34B02C01A5241030A8B423C
:1092B00001D30B02C01A5241CDD2C3098B4201D354
:1092C000CB01C01A524183098B4201D38B01C01AD2
:1092D000524143098B4201D34B01C01A5241030949
:1092E0008B4201D30B01C01A5241C3088B4201D3F8
:1092F000CB00C01A524183088B4201D38B00C01AA5
:10930000524143088B4201D34B00C01A5241411ACB
:1093100000D20146524110467047FFE701B50020D8
:1093200000F0F0F802BDC0460029F7D076E770479C
:1093300003460B437FD4002243088B4274D30309B6
:109340008B425FD3030A8B4244D3030B8B4228D357
:10935000030C8B420DD3FF22090212BA030C8B427D
:1093600002D31212090265D0030B8B4219D300E01D
:10937000090AC30B8B4201D3CB03C01A5241830BA2
:109380008B4201D38B03C01A5241430B8B4201D352
:109390004B03C01A5241030B8B4201D30B03C01A7B
:1093A0005241C30A8B4201D3CB02C01A5241830AF5
:1093B0008B4201D38B02C01A5241430A8B4201D324
:1093C0004B02C01A5241030A8B4201D30B02C01A4E
:1093D0005241CDD2C3098B4201D3CB01C01A5241B5
:1093E00083098B4201D38B01C01A524143098B423E
:1093F00001D34B01C01A524103098B4201D30B0127
:10940000C01A5241C3088B4201D3CB00C01A52414B
:1094100083088B4201D38B00C01A524143088B4210
:1094200001D34B00C01A5241411A00D201465241A9
:10943000104670475DE0CA0F00D04942031000D3C8
:109440004042534000229C4603098B422DD3030A1D
:109450008B4212D3FC22890112BA030A8B420CD32D
:10946000890192118B4208D3890192118B4204D356
:1094700089013AD0921100E08909C3098B4201D3D6
:10948000CB01C01A524183098B4201D38B01C01A10
:10949000524143098B4201D34B01C01A5241030987
:1094A0008B4201D30B01C01A5241C3088B4201D336
:1094B000CB00C01A524183088B4201D38B00C01AE3
:1094C0005241D9D243088B4201D34B00C01A5241BA
:1094D000411A00D20146634652415B10104601D347
:1094E0004042002B00D54942704763465B1000D3D1
:1094F000404201B5002000F005F802BD0029F8D077
:1095000016E770477047C0468446101C62468C467A
:10951000191C634600E0C0461FB501F02FF9002872
:1095200001D40021C8421FBD10B501F089F84042A6
:10953000013010BD10B501F021F9002801DB002039
:1095400010BD012010BDC04610B501F017F900286C
:1095500001DD002010BD012010BDC04610B501F096
:10956000A9F8002801DC002010BD012010BDC04674
:1095700010B501F09FF8002801DA002010BD01208D
:1095800010BDC0469E2110B5C905041C02F090F81C
:10959000002803D1201C00F0A9F910BD9E21201C39
:1095A000C90500F007F800F0A1F980231B069C46CE
:1095B0006044F2E7F0B54F46D64646464400C0B593
:1095C000C20F47024802400A844666467B0A4800AA
:1095D000C90F9A46240E1500DB00000E8946F600DE
:1095E000FF2800D18FE001214F464F4039009142C2
:1095F00066D0221A002A00DC9DE000283DD1002E12
:1096000000D18BE0511E002900D0B5E001249B1B46
:109610005A0144D59B019F09380002F053F80538E0
:109620008740844200DD96E0041B3A00202001348C
:10963000E240041BA7403B005F1EBB4100241343D4
:109640005A0704D00F221A40042A00D004335A01CA
:1096500027D50134FF2C00D179E001229B015B0A60
:10966000E4B22A405B02E405580AD20720431043C3
:109670001CBC90469946A246F0BDFF2CE0D080214C
:10968000C9040E431B2A7BDC31002020D140821A02
:109690009640721E96410E439B1B5A01BAD45A073C
:1096A000D0D10122DF082A40FF2C33D1002F00D176
:1096B000A8E08023DB033B435B025B0AFF24D1E786
:1096C000211A00294CDD00282AD0FF2CB8D0802098
:1096D000C00406431B2900DDAFE030002027C8404E
:1096E000791A8E40711E8E4106439B195901D6D5B9
:1096F0000134FF2C00D185E001227A491A405B0831
:109700000B4013439CE7002E00D070E76BE73B1E35
:10971000C5D100227B025B0AE4B2A3E714008FE705
:10972000002E4DD0481E002857D19B1901245A0104
:10973000B5D50224E0E7002A25D1621CD2B2012A65
:1097400072DD9F1B7A0135D5F71A0D0064E70122FF
:1097500000232A4086E73B00634A241A13406FE740
:1097600000296CD1611CC8B201284EDDFF2949D007
:109770009B195B080C0063E7FF2A41D00A0081E7D0
:1097800001269B1B89E7002C1CD0FF2821D08024B8
:10979000E404524223431B2A00DD96E01C002025EE
:1097A000D440AA1A93405A1E93412343F31A04004B
:1097B0000D002DE7002F00D02EE700220024A9E79E
:1097C0000C003DE7002B58D0D243002AEED0FF28F2
:1097D000E1D13300FF240D0032E7FF2910D0010052
:1097E00078E7002B6ED0FF24002E00D128E78022DE
:1097F0005146D203114203D06146114200D13300D9
:10980000FF241DE7FF2400232CE7002CE9D1002BC7
:1098100063D0002E00D113E79B195A0100D43EE714
:10982000314A0C0013400BE7002C1ED1002B2FD126
:10983000002E4FD033000D0002E7012655E7002C23
:109840001FD1002B43D0C94300290BD0FF2839D0AA
:109850001B2944DC1C002027CC40791A8B40591E60
:109860008B4123439B19040040E7002B1AD1002EA3
:1098700024D180270022FF031BE7330004000D00E2
:10988000DEE6FF281ED08024E40449422343DFE7BC
:10989000002E00D1D4E69F1B7A0100D437E7F31ADB
:1098A0000D00CDE6FF24002E00D1C9E680225046EF
:1098B000D2031042A4D060461042A1D133000D0063
:1098C000FF24BDE63300FF24BAE601236EE7330030
:1098D0000400B5E6002700221CE73300B0E60123B0
:1098E000C0E7C046FFFFFF7DFFFFFFFB41024300D3
:1098F000C20F490A1B0E00207E2B0DDD9D2B0CDCB8
:10990000802000040143952B0ADC9620C31AD9401D
:109910004842002A00D108007047034BD018FBE7EB
:10992000963B9940F4E7C046FFFFFF7F10B5041E49
:1099300027D001F0C7FE9E231B1A962B0ADC962225
:10994000D21A94406402640ADBB26402DB05600A46
:10995000184310BD992B17DC9922D21A002A27DD53
:1099600094402200134C1440510704D00F210A40A8
:10997000042A00D00434620112D4A401640ADBB2C8
:10998000E3E700230024E0E7B9222100D21A914046
:109990000A00511E8A410521091ACC401443DBE715
:1099A000044B1C409F23A4011B1A640ADBB2CCE7C2
:1099B0002200D7E7FFFFFFFBF8B54546DE465746D6
:1099C0004E460C03E0B54E00C90F88460D00610AF3
:1099D000440F0C43C70019035800DB0F9B464B0A8A
:1099E000510F0B43760D400D1900D200D84500D120
:1099F000AEE0351A002D00DCF6E000280FD113434D
:109A000000D1DBE06B1E002B00D037E1BA1A974281
:109A1000BF41641A7F42E41B0126170024E0C64BB5
:109A20009E424DD080231B041943382D00DD07E1F1
:109A30001F2D00DD38E12020431B9A460B005046C5
:109A40008340994613004846EB40184303005046B4
:109A50008240501E8241E9401A43BA1A611A974265
:109A6000A441170064420C1B230262D56402650AFC
:109A7000002D00D1DFE0280001F024FE0300083BA8
:109A80001F2B00DDD2E020223C00D21A9D40D440A2
:109A90009F4025439E4200DDC4E09E1B731C1F2B8C
:109AA00000DDF1E0202238002900D21AD840914090
:109AB00097402C000143781E8741DC4000260F436D
:109AC0007B0709D00F233B40042B05D03B1DBB4235
:109AD000BF417F42E4191F0023022CD5964B01366B
:109AE0009E4200D19AE04546944BFF081C40600717
:109AF000760564020743240B760D00212403230B13
:109B00000C0D8F4A24051C431440330523435B008E
:109B1000ED075B082B43380019003CBC9046994682
:109B2000A246AB46F8BD6446044300D111E20400EE
:109B300067467B07C6D145466007FF080743E40830
:109B40007D4B9E4230D024037605240B760DD4E75E
:109B5000331A9A46002B78DD002831D076488642A9
:109B6000AED08020000401435346382B00DCE9E0EE
:109B70000A43511E8A410021D219BA42BF41091934
:109B80007C4217000C192302D3D56B4B01369E4241
:109B900000D13AE10120694B1C407B0807401F437C
:109BA000E007074364088BE723003B4300D1CBE188
:109BB0008022120314432403240B9EE72E007FE728
:109BC0000800104300D1B4E0581E002800D0DEE0A9
:109BD000BA18BA429B4164185B42E4181700012688
:109BE0002302A6D50226D5E7002D6ED1701C4005B4
:109BF000400D012800DCF9E0B81A84468742804114
:109C0000E51A40422D1A280200D489E0D71BBA4237
:109C100092411C1B5242A51AD84629E7454600240A
:109C200000276AE7454CF61A2C4049E73D002838E2
:109C3000854000272EE7380001F044FD20301DE765
:109C40000A43511E8A41002107E7002B00D0F3E0B0
:109C5000701C43055B0D012B00DCADE0364B9842D8
:109C600000D1D1E0BA18BA42BF4164187F42E4196A
:109C7000E707520817436408060021E72E4885428B
:109C800000D193E01D00D0E629001F3EF140202BBB
:109C900000D18DE04022D31A9D402F437D1EAF415D
:109CA00000240F43002644E72B000800203BD84047
:109CB0000300202D00D17DE04020451BA9400A4330
:109CC000511E8A4100211A43C7E6002E50D01A4E79
:109CD000B04257D080266B429946360434434B46F7
:109CE000382B00DDD6E01F2B00DD35E12026F51AEC
:109CF0002600AE40B2463E00DE40AC463500564639
:109D00002E436546AF407D1EAF41DC403743D71B35
:109D1000BA4292410C1B5242A41A0600D846A3E64E
:109D2000644667462C4300D0A2E6002500260027A3
:109D300006E71E00C4E6C046FF070000FFFF7FFFE6
:109D4000FFFF0F801F2B63DC2020C31A0800984000
:109D50009C46834653461000D8400300584618439B
:109D600063469A40531E9A4153460243D94003E743
:109D700026003E4306D0EB439946002BC7D0944EB5
:109D8000B042ACD10C0017000600D84698E6904BC4
:109D90009A450BD08246E7E6002800D09EE01800E6
:109DA000104300D1E9E01C001700D846884E87E632
:109DB000002572E7002182E723003B43002E00D0FC
:109DC000ABE0002B00D1E7E00B00134300D177E6B6
:109DD000BA18BA42BF4164187F42E419230200D482
:109DE000F2E07C4B17001C40060069E62000384377
:109DF000002ED1D100285BD11C00144300D1A8E073
:109E00001C001700D8465BE606000024002797E6F2
:109E100050460B002038C34099465346202B00D1B2
:109E200095E0402350461B1A99400A43511E8A412F
:109E30004B4600211A439FE6002E30D126003E43B8
:109E400067D0DB439A46002B1CD0614EB04260D0F5
:109E50005346382B00DD96E01F2B00DD9FE02026C7
:109E6000F31A26009E409C46B34653463E00DE4011
:109E700033005E461E4363469F407B1E9F41534610
:109E8000DC403743BF189742924164185242A418ED
:109E9000060078E627437C1EA741002437E74C4E96
:109EA000B04236D080265B4236049A463443CFE730
:109EB0001800104300D103E6B81A84466745AD4147
:109EC000E01A6D42401B050200D42CE6D71BBA42B3
:109ED00092411C1B5242A41AD846F1E518001043C7
:109EE00000D163E7F808670707438020E408000310
:109EF000044208D0DD08054205D1D20859071143B4
:109F00000F002C00D8467B0FE4001C43FF00304EAE
:109F1000D6E50C0017000600D2E5002B38D00B0068
:109F2000134300D142E7F808670707438020E4089D
:109F300000030442E7D0CB080342E4D1D20849072A
:109F400011430F001C00DEE700270024D5E50021A7
:109F50006BE700250027F3E54E462500203EF5403F
:109F60004B462E00202B2DD04025ED1AAC40274328
:109F70007C1EA74100243743C9E680240025240322
:109F8000134E0027DCE527437C1EA741002479E718
:109F90000C0017000E4E93E50C00170090E5564696
:109FA0002300203EF34099465346202B0ED04023F9
:109FB00056469B1B9C4027437C1EA7414B460024D2
:109FC0001F435FE70024D2E71700B2E50024F2E761
:109FD000FF070000FFFF7FFFF0B557464546DE460E
:109FE0004E46E0B54C000E0387B0834692461D00F6
:109FF0008046360B640DCF0F002C4FD06F4B9C4228
:10A0000035D08023420F1B04F60013433343994697
:10A01000C30098466A4B00269C4600236444039381
:10A020002B031B0B9B466B00ED0F50465B0D019500
:10A030005ED0624A934253D05A46D1008022400FEC
:10A04000120402430A4393465246D1005C4A9446A6
:10A05000002263443800684084460290E41A1643A4
:10A060000F2E00D9B4E0574BB6009B599F46030012
:10A07000334399466CD10023984602330826039354
:10A08000CEE7CB464146039A0197022A65D1019B50
:10A090004A4C9C460023002298466BE00300334361
:10A0A00099464ED0002E00D1BCE1300001F00AFBF1
:10A0B00003000B3B1C2B00DDACE11D22D31A5A46DA
:10A0C0000100DA4008398E401300334399465B465D
:10A0D0008B40984600233C4C0026241A03939FE7AC
:10A0E00051465A46114329D1002293460232B1E724
:10A0F000594601431ED05B46002B00D19EE15846D5
:10A1000001F0E0FA03000B3B1C2B00DD8FE10200A5
:10A110005946083A91408B461D21CB1A5146D940E9
:10A120000B0059460B4351469B469140264B00225B
:10A130001B1A8FE7002301229B468BE7514603221F
:10A1400088E700239846013304260024039367E739
:10A150000323B14603930C2662E7032A00D15CE295
:10A16000019B012A00D0E4E113409C460023002417
:10A170000022984600211203130B0A0D12051A4300
:10A180002305124C40462240134362465B00D2072F
:10A190005B081343190007B03CBC90469946A246A1
:10A1A000AB46F0BD002380229C4612039846034C28
:10A1B000E0E70023014C00229846DBE7FF070000A0
:10A1C00001FCFFFFA4BF00000DFCFFFFFFFF0F809D
:10A1D000D94500D939E100D134E1002346464D4646
:10A1E0009A46013C5B460A0E1B021A430B02170CEF
:10A1F000039313041B0C3900280090460193FFF7CA
:10A200000DF80200019B83465A432800390091460D
:10A21000FFF78AF8350C09040D43A9450DD95B46B3
:10A220004544013BA84500D93AE1A94500D837E1AA
:10A2300002235B429C464544E3444B46EB1A3900FB
:10A2400018000493FEF7EAFF019B05004343390021
:10A2500004989946FFF768F8330409041B0C0B4374
:10A26000994509D943446A1E984500D91AE1994590
:10A2700000D817E1023D43444A469B1A5A4612044D
:10A280002A4303999346100C0A0C914609045A4636
:10A29000090C4E460D001204120C45430591514322
:10A2A0007243704352190E0CB218954203D980259F
:10A2B0006D02AC466044150C09041204090C281800
:10A2C0005218834200D2CEE000D1C8E01D1A534696
:10A2D0009E1AB24592415242AB1A9A46984500D115
:10A2E00017E139001800FEF799FF019B0500434371
:10A2F000390050460493FFF717F804980B04310C0B
:10A300001943884209D941446B1E884500D907E1A9
:10A31000884200D804E1023D4144049BCB1A180056
:10A3200039000493FEF77AFF019B824643433900CC
:10A3300004980193FEF7F8FF01980B043104090C0F
:10A34000194388420DD953464144013B884500D901
:10A35000E8E0884200D8E5E002235B429C464144A5
:10A36000E244019B2D04CE1A51462943059D4F46D8
:10A370002A000B04080C1B0C5A4345437B437843CB
:10A380005B19170CFB189D4203D980256D02AC4662
:10A3900060441D0C12041B04120C28189B188642E2
:10A3A00000D293E000D18EE001231943A04BE318C3
:10A3B000002B00DC99E04A0700D09EE05A46D2010B
:10A3C00006D55A469B4B1A4080239346DB00E31880
:10A3D000994A934268DD0123029A984C1A4000235F
:10A3E000944698460022C5E680224B46120313424B
:10A3F0000AD05B46134206D11A431203120BAC4635
:10A4000088468E4CB6E64B461A431203120BBC46E6
:10A410008A4CAFE603005A46283B9A4000239146F7
:10A42000984657E6584601F04DF9203040E60300C3
:10A430005246283B9A400021934677E601F042F9C4
:10A4400020305FE6884500D2C7E64B46DE075D0850
:10A4500043465B081E434346DB079A46C2E6002597
:10A46000924500D333E7039E5946B446E244B245D1
:10A47000AD416D424544EB180139984507D29842E9
:10A4800000D97FE000D1BCE01D1A8B461FE798453C
:10A49000FAD1039D5545F2D943468B461D1A16E75E
:10A4A0009B46CAE61500E7E65A46C90852070A4322
:10A4B0005B0590465C0D5A460123029952021940F1
:10A4C000120B8C4656E6002B00D16FE746444A1E1D
:10A4D000B04529D91100864200D065E7039A93421E
:10A4E00000D061E762E7012149420120C21A382AFF
:10A4F00021DD029B03409C4638E60F220A40042AD5
:10A5000000D15BE70A00111D9142924152429344EF
:10A5100054E7474BE318002BE5DD01225242F2E7F6
:10A520001D00FAE69A461CE7B04239D86ED01100F9
:10A530003AE702933AE71F2A3CDC20239B1A0C00DF
:10A540005846994098404B1E99415B46D440D340B1
:10A55000204308431A00430709D00F230340042B6C
:10A5600005D00100081D88429B415B42D2181302AE
:10A570003AD50123029A01241A40002394469846B2
:10A580000022F7E5022149428C46039DE344AC4694
:10A59000E244AA45AD416D424544ED182D1A96E6B8
:10A5A0008A1E03994D008D428941494241447618E3
:10A5B00003958FE71F204042C31A5846D840030036
:10A5C000202A28D040205D46821A954029434A1E01
:10A5D00091411943072300220B4009D00F23002289
:10A5E0000B400800042BBDD1010053075202120B8F
:10A5F000C9081943012388460299002419408C4652
:10A60000B8E55245BED88B46002560E6039D9D42C5
:10A61000C6D3110062E70025D8E780225B4612030B
:10A620001A43019B1203120B9C468846034CA1E57A
:10A63000FF030000FFFFFFFEFE070000FF07000012
:10A64000F0B54F464646D6465C00C0B51F03DB0F4B
:10A650009A46174B0E034D0084468046360B6D0D0F
:10A66000C90F91463F0B640D01209D4208D09C42CA
:10A6700001D0A5420BD01CBC90469946A246F0BD25
:10A6800063463343F7D1AC42F5D13A43F3D10120CD
:10A69000BE42F0D1C845EED1514507D0002DEAD1D8
:10A6A00063461E433000461EB041E4E70020E2E767
:10A6B000FF070000F0B54546DE4657464E46E0B57A
:10A6C0001F033D0B2C4F0E034C00AB465D00844630
:10A6D000360B640DC90F90466D0DDB0FBC422AD0BE
:10A6E000254FBD422DD0002C0FD1304307008146AD
:10A6F00078427841C0B2002D17D15F463A4314D159
:10A700004B460020002B0AD006E0002D02D158460F
:10A71000024301D0994218D04842012108433CBC71
:10A7200090469946A246AB46F0BD0028F2D00120E3
:10A73000013B1843F3E737000743D1D002204042E2
:10A74000EDE75F461743CED0F8E7AC42E4DC03DA2E
:10A75000481E01210843E2E75E45DDD806D000200F
:10A760005E45DCD20123481E1843D8E7C445D3D840
:10A770000020C445F6D3D2E7FF070000F0B54E46EF
:10A780004546DE4657465C00E0B51F03DB0F9946A1
:10A790002A4B0E034D00C90F8446360B6D0D8B46B8
:10A7A00090463F0B640D9D4220D0244B9C4222D00A
:10A7B000002D12D1304343424341DBB2002C1FD065
:10A7C000002B0CD04B460120013B034318003CBC3E
:10A7D00090469946A246AB46F0BD002C16D0CB451C
:10A7E00017D05B46594201230B43EFE731000223A8
:10A7F0000143EBD1D9E7390002231143E6D1D7E772
:10A800003A43DDD100230028E0D0EAE73A43E6D11D
:10A81000E7E7A542E5DC05DBBE42E2D807D000232E
:10A82000BE42D3D25946012301390B43CEE7C4457A
:10A83000D7D80023C445F5D3C8E7C046FF070000BA
:10A84000F0B557464546DE464E46E0B50C03984601
:10A850004E00230B87B0070092469B46760DCD0F26
:10A86000002E6BD06D4B9E4235D080245B46420F4C
:10A870002404DB0014431C43C3009946684BA346E1
:10A880009C46002300276644029343461C035A005B
:10A89000DB0F5046240B520D984600D176E05F4BFB
:10A8A0009A426DD08023410F1B040B435C49E400A6
:10A8B0008C461C43C300002062444146B6186940E0
:10A8C000721C0191944607430F2F00D9B0E0554AFE
:10A8D000BF00D25997465B460343994600D087E0B4
:10A8E00000239B46023308270293CEE7424601929B
:10A8F000022867D0032800D10EE2012800D062E1CF
:10A90000002300240022994601990140CDB2002184
:10A9100012030B0D120B1B051343434A240513406E
:10A920001C436400ED0764082C434846210007B02F
:10A930003CBC90469946A246AB46F0BD03439946BF
:10A940004FD05B46002B00D189E1584600F0BAFE9B
:10A9500003000B3B1C2B00DD7AE11D22D31A3A00C9
:10A9600001005C46DA4008398C4013008F402343D5
:10A970009B46B94600232D4E0027361A029384E7E2
:10A98000534623432AD10024022096E7534623430B
:10A9900020D0002C00D157E1200000F093FE0300EE
:10A9A0000B3B1C2B00DD49E11D21CB1A5146020057
:10A9B000D9405346083A944093400C431B4A121A1C
:10A9C00000207AE70125019B144C1D400023002242
:10A9D00099469CE70024002201206EE7534603209D
:10A9E0006BE700239B4601330427002602934CE7C4
:10A9F000032381460C27029347E78022002300258A
:10AA000012039946054C82E75C464B4602986FE775
:10AA10005C464B46019502986AE7C046FF07000076
:10AA200001FCFFFFE4BF0000FFFF0F800DFCFFFFF4
:10AA30004A464946170C1A0C1B041B0C0804190043
:10AA4000000C41431500884619007D437943039566
:10AA500089462900150045434D44029545462D0C75
:10AA6000AA46029D5544A94506D98A468021490235
:10AA70008946CA4451460391290C04914146090470
:10AA80002D04090C88462900250C24044144240C7B
:10AA90000591210041438846210079438A46684355
:10AAA000414650448146080C48446F43824503D9CF
:10AAB0008021490289464F44010C894639004944A6
:10AAC000029141460F0404993F0C88460004C019C6
:10AAD00080444146049159460F0C0904090C8846EC
:10AAE00059438A4639005143894641464A435146B3
:10AAF000090C8B467B43D2185A44934203D98023D6
:10AB00005B029B46D94451460904090C8A464146DA
:10AB100061437C43130C12044B445244A1468A46C1
:10AB20003C0041466C434D4351464D440F0C7D194A
:10AB3000A94503D98021490288464444049F0399CA
:10AB4000B84641448B468345804141428846514640
:10AB500008042F04000C3F18584602991018894623
:10AB6000904292414F44BA46524299469346C2445B
:10AB7000D144CB448F42BF41C245894199459B4155
:10AB8000934592417F4249422D0C52420F435B4212
:10AB900013437F19FF185B463C19DB0D059A6402CD
:10ABA0001C43430213435D1EAB415A46C00D034391
:10ABB00052021343E20156D501205A0803401343C1
:10ABC000E207134364085A48604400284DDD5A07E1
:10ABD00009D00F221A40042A05D01A1D9A429B411F
:10ABE0005B42E4181300E20104D58020514AC00002
:10ABF00014406044504A904200DDE3E60125DB0842
:10AC000062071A436402019B9146220B4405640DBE
:10AC10001D407CE6802259461203114208D014429E
:10AC200006D122431203120B45469946434C6EE669
:10AC30005B461A431203120B404C68E6030054466D
:10AC4000283B9C400023B9E600F03CFD2030A6E6FE
:10AC50000300283B9F400023BB4699468AE600F04C
:10AC600031FD203074E6B446ADE701252A1A382AB2
:10AC700006DD019B00241D4000230022994646E684
:10AC80001F2A21DC20252000AD1A1E00AB40A84061
:10AC9000D6405D1EAB4130431843D440430709D032
:10ACA0000F230340042B05D00300181D98429B413D
:10ACB0005B42E418230221D50125019B01241D409C
:10ACC00000230022994622E61F2521006D42281A02
:10ACD000C1400800202A1DD05F35AA1A94402343A2
:10ACE0005C1EA341072503431D400022002D09D00F
:10ACF0000F2200241A401800042AD6D10300650749
:10AD00006402220BDB082B4301259946019B00249A
:10AD10001D40FCE50024E2E78022012512032243C6
:10AD200001991203120B0D409946044CEFE5C04601
:10AD3000FF030000FFFFFFFEFE070000FF0700000B
:10AD4000F0B54646D6464F460C03C0B5CD0F4E0073
:10AD5000610A440F0C43C1005800400D84468A46E6
:10AD60000F001903500F490A0143C648760DA84643
:10AD7000DB0FD200844500D1D8E001204340AB4234
:10AD800000D1A6E06046351A002D00DC05E1002860
:10AD900010D10B00134300D1D7E06B1E002B00D065
:10ADA0004BE153469F1ABA458041641A4042241A27
:10ADB00001261EE0B34B9E4248D080231B0419435A
:10ADC000382D00DD19E11F2D00DD4CE120230F009F
:10ADD0005B1B10009A409F40E840531E9A41E94097
:10ADE000074317435346DF1B611ABA45A441644227
:10ADF0000C1B230200D4C5E06402650A002D00D1BB
:10AE0000F6E0280000F05EFC0300083B1F2B00DD8D
:10AE1000E9E020223C00D21A9D40D4409F402543C7
:10AE20009E4200DDDBE09E1B731C1F2B00DD0AE150
:10AE300020223800D21A290097402C009140D84097
:10AE40007A1E9741DC40002601430F437B0709D05F
:10AE50000F233B40042B05D03B1DBB42BF417F422B
:10AE6000E4191F00230225D5864B01369E4200D1EE
:10AE7000AFE0854B01251C4043466207FF08640292
:10AE800076051743240B760D1D4000212403230B68
:10AE90000C0D7E4A24051C431440330523435B00FC
:10AEA000ED075B082B43380019001CBC90469946FF
:10AEB000A246F0BD012543466207FF081743E40898
:10AEC0001D40704B9E4236D024037605240B760D30
:10AED000DBE76346F31A002B00DC94E060460028B1
:10AEE00035D068488642B1D080273F043943382B9B
:10AEF00000DCFDE00A43170000217A1E9741574409
:10AF000057458041091944420C1923023AD55D4B3B
:10AF100001369E4200D14BE101225B4B1C407B0875
:10AF200017401F43E207174364088FE708001043E8
:10AF300000D024E721E723003B4300D1B9E1802280
:10AF4000120314432403240B9FE72E007EE708001E
:10AF5000104300D1CAE0581E8446002800D0E7E024
:10AF6000524452458041641840422418170001267B
:10AF7000230207D50226CFE764462C4300D1B3E174
:10AF80002C0067467B0700D062E76307FF081F437A
:10AF900001254346E4081D4093E7002D78D1751C38
:10AFA0006D056D0D012D00DCF2E05046801A8245E2
:10AFB000BF41651A7F42ED1B8446280200D48CE015
:10AFC0005046171ABA4292410C1B5542651B9846CF
:10AFD00014E70125434600241D40002755E72A4C6D
:10AFE000F61A2C4032E73D0028388540002717E745
:10AFF000380000F067FB203006E70A431700002105
:10B000007A1E9741EEE6002B00D0E5E0731C9C46CB
:10B010005B055B0D012B00DC9FE01A4B9C4500D1CA
:10B02000C5E0524452458041641840422418E70765
:10B03000520817436408664608E71248854200D163
:10B0400085E01D00BCE629001F3EF140202B00D109
:10B050007FE04022D31A9D402F437D1EAF41002444
:10B060000F4300268EE72B000F00203BDF40202DF2
:10B0700071D040235D1BA9400A43511E8A41002123
:10B080001743AFE6FF070000FFFF7FFFFFFF0F80C2
:10B09000002E3ED0B34EB44545D0802636046D42D6
:10B0A0003443382D00DDA8E01F2D00DD1FE12026F0
:10B0B00027005046761BB740E84007435046B04053
:10B0C000461EB041EC403843171ABA4292410C1B5D
:10B0D0005242A41A664698468BE6644667462C435D
:10B0E00000D08BE6002500260027EAE61E00ADE62C
:10B0F0001F2B60DC2027F81A0F00844687401000C1
:10B10000D840074360468240501E8241D9401743D1
:10B11000F5E626005046064305D0ED43002DD3D07A
:10B12000904EB445BDD10C001700664698468DE69A
:10B130008C4883420BD06346D9E6002D00D096E0C0
:10B140000800104300D1E2E00C0017009846854E3D
:10B150007CE6002580E700218EE72300504603436C
:10B16000002E00D0A8E0002B00D1DEE00B0013433E
:10B1700000D16BE652445245804164184042241885
:10B180001700230200D4FDE6774B66461C405DE6BF
:10B19000250050460543002ECFD1002D4FD10C0085
:10B1A000144300D1A0E00C00170098464EE6664616
:10B1B0000024002785E61F000800203FF840070014
:10B1C000202B00D18EE04020C31A99400A43511E23
:10B1D0008A410021174392E6002E14D126005046E2
:10B1E000064362D0DB43002B5CD187189742924123
:10B1F00064185242A418664687E650462043441E0F
:10B20000A041002460E7574EB4454ED08026360456
:10B210005B423443382B00DD7FE01F2B00DD8BE0E9
:10B22000202627005046F61AB740D840074350461C
:10B23000B040461EB0410743DC40BF18D6E70D00C2
:10B24000154300D102E65046801A8245BF41651A77
:10B250007F42ED1B8446280200D48DE65046171A23
:10B26000BA4292410C1B5242A41A9846EEE50D00D8
:10B27000154300D16BE750466707C008074380209D
:10B28000E4080003044207D0CD08054204D12C0095
:10B290009846D70849070F437B0FE4001C43FF0083
:10B2A000304ED3E52F4EB445B4D10C00170066469E
:10B2B000CCE500270024E8E5002B39D00B00134330
:10B2C00000D144E7C008670707438020E408000373
:10B2D0000442E1D0CB080342DED1D70849070F432F
:10B2E0001C00D9E7002171E700250027E9E52E00C1
:10B2F0002700203EF740202D2FD04026751BAC4064
:10B3000050462043441EA04100243843DCE68024FC
:10B3100000252403134E0027D3E5504620430700A1
:10B32000781E87410024BF1860E70C0017008DE5E8
:10B330000C0017000B4E89E51E002700203EF74049
:10B34000202B0CD04026F31A9C4050462043441E2C
:10B35000A04107430024BF1848E70024D0E7002499
:10B36000F3E7C046FF070000FFFF7FFF70B50E4EFA
:10B370000D031C0349005B002D0B490D240B5B0DD5
:10B38000B14204D0084900208B4208D070BD05436B
:10B390000120002DFAD1044900208B42F6D114433C
:10B3A0002000441EA041F1E7FF07000030B5134D17
:10B3B0000A034B00120B5B0DC90F0024AB4210DDDA
:10B3C0000F4CA3420FDC80240E4D64032243ED1A80
:10B3D0001F2D0BDD0C48C31ADA405442002900D15E
:10B3E0001400200030BD094BCC18FAE7084CE840A7
:10B3F000A44663449A400243EFE7C046FE030000C0
:10B400001D0400003304000013040000FFFFFF7F51
:10B41000EDFBFFFF70B5002830D0C317C4185C40A7
:10B42000C50F200000F04EF9174B184A1B1AD21A0C
:10B430001F2A18DD164AD21A9440002224035B0505
:10B44000240B5B0D0021100024030A0D240B1205B0
:10B450002243104C1B05224013435B00ED075B08A1
:10B460002B43190070BD210091400A000B21081ADE
:10B47000C4405B052403240B5B0DE3E70025002398
:10B4800000240022DEE7C0461E0400003304000052
:10B4900013040000FFFF0F804100090E4B1C70B524
:10B4A000DBB24602750AC40F012B14DDE0239B00BA
:10B4B0006D07360BCB1800210A0D280012051C4D14
:10B4C00032435B052A405B0813435B00E4075B08DB
:10B4D0002343190070BD002914D1002D1ED028006F
:10B4E00000F0F0F80A281CDC0B232A001B1ADA40B3
:10B4F000030015339D400F4B12031B1A5B05160BFF
:10B500005B0DD8E7002D06D0320B802636036D0781
:10B510001643094BCFE7084B0026CCE70023002653
:10B52000C9E703002A000B3B9A400025E3E7C04629
:10B53000FFFF0F8089030000FF070000F0B54C00FB
:10B54000640D0B03621C450F5B0A52052B43C90FA8
:10B55000C500520D012A28DD3A4AA618FE2E1BDC32
:10B56000002E3EDD80010200501E82416D0F2A43F5
:10B57000DB0013435A0704D00F221A40042A00D0DC
:10B5800004338022D2041A405AD00136FF2E03D051
:10B590009B015B0AF4B201E0FF2400235802E4059A
:10B5A000400AC90720430843F0BD002C07D01D43C3
:10B5B000F2D08020DB0080040343FF26DAE72B4330
:10B5C00003D00523DB08FF2C03D05B025B0AE4B247
:10B5D000E4E7002B32D08020C00303435B025B0A08
:10B5E000DCE73200173214DB80221E2712041343DB
:10B5F000BF1B1F2F0FDC144A944664442A00A54049
:10B600002E00A340751EAE41FA403343134300267B
:10B61000B0E70024D5E702225242961B1A00F240FE
:10B62000202F09D0094884466444A3402B435D1E63
:10B63000AB41002613439DE70023F7E70023ADE766
:10B640003400BFE780FCFFFF82FCFFFFA2FCFFFF8E
:10B650008446081C6146FFE71FB500F0B7F80028D4
:10B6600001D40021C8421FBD10B500F049F8404286
:10B67000013010BD10B500F0A9F8002801DB002052
:10B6800010BD012010BDC04610B500F09FF8002885
:10B6900001DD002010BD012010BDC04610B500F036
:10B6A00055F8002801DC002010BD012010BDC04667
:10B6B00010B500F04BF8002801DA002010BD012081
:10B6C00010BDC0461C2101231B04984201D3000C6D
:10B6D00010391B0A984201D3000A08391B09984205
:10B6E00001D30009043902A2105C40187047C0461B
:10B6F000040302020101010100000000000000003B
:10B7000070B5420045024E024C00C30F6D0A120E86
:10B71000760A240EC90F0120FF2A06D0FF2C03D081
:10B72000A24201D1B54206D070BD002DFCD1FF2C44
:10B73000FAD1002EF8D18B4206D00120002AF3D195
:10B740002800451EA841EFE70020EDE7F0B54200D4
:10B7500045024C02C30F48006D0A120E640A000E27
:10B76000C90FFF2A1ED0FF2821D0002A0AD16E421D
:10B770006E41F6B200280FD1002C0DD10020002D13
:10B7800009D005E0002801D1002C01D08B4211D056
:10B79000012158420843F0BD002EF7D001200139A5
:10B7A0000843F8E7002DDED002204042F3E7002CEA
:10B7B000DBD0F9E78242EBDC04DBA542E8D80020CD
:10B7C000A542E8D20121581E0843E4E7F0B5420043
:10B7D0004D024C004602760A120EC30F6D0A240E6B
:10B7E000C90FFF2A16D0FF2C18D0002A0AD17042A8
:10B7F0007041C0B2002C15D0002805D001200139BD
:10B800000843F0BD002C13D0994214D001205B42B4
:10B810001843F6E70220002EF3D1E4E70220002DC2
:10B82000EFD1E2E7002DE7D10020002EE9D0EDE7CF
:10B83000002DE9D1EAE7A24206DCDFDBAE4203D805
:10B840000020AE42DAD3DCE7012049420843D8E7C2
:10B85000002103E00A4B5B584350043109480A4B6E
:10B8600042189A42F6D3094A02E0002313600432D8
:10B87000074B9A42F9D3FDF7E7FB00F00BF870474E
:10B8800058C0000000F0FF1F94F0FF1F94F0FF1F4E
:10B8900078FAFF1F02211F4A10B553688B4353608B
:10B8A00062B6F6F70BFFF6F70BFEF6F7F5FFFBF7C0
:10B8B00045FAFBF797FCF7F78BF8F7F7EDF8164C1E
:10B8C000002808D0F7F7E8F82070F7F7E5F8FF232D
:10B8D000A08263706382A078F6F756FEE078F6F7F0
:10B8E000D1FEE28AA18A207CFDF772FAFCF735F9D5
:10B8F000FDF706FAFCF780FDF8F734F9FBF7DEFFF9
:10B900008022064B9A60FAF769FFFBF7C3FCFBF74E
:10B91000D6FFF8E70080044004F0FF1F40F00F401E
:10B92000002310B59A4200D110BDCC5CC454013341
:10B93000F8E70000F0B5C64600B58CB004000D0075
:10B9400000F080F83A4B06001B780F005BB2984677
:10B9500001330FD022002B0020002900FFF706FD45
:10B96000002807D10022002320002900FDF7F6FD62
:10B97000002805D0300039000CB004BC9046F0BD62
:10B980002C4B0A900393434604940595069407951F
:10B99000002B1AD1E022284B1206089209932000AE
:10B9A000002200232900FDF7BFFD002838D0022324
:10B9B000029302A800F048FA002817D00A9B0193CE
:10B9C000002B18D1089E099FD4E700221B4B2000B2
:10B9D00008920993290000220023FDF7A5FD002805
:10B9E0000FD0022302934346022BE2D100F034FA37
:10B9F00022230360E2E700F02FFA0A9B0193036021
:10BA0000E0E7012302934346022B0BD100F024FA16
:10BA1000212303600A4800F019FA08900991CDE744
:10BA20000123029302A800F00FFA0028F2D1EDE7FB
:10BA30008CF0FF1F30C00000FFFFEFC70000F0FFD9
:10BA400034C00000F0B5D6464F464646C0B5DA4A87
:10BA500088B00B00914255DC4A005208024300D1E5
:10BA6000EFE0002900DA79E1D44B0022FEF7E8FE8E
:10BA70003625D34C0B006D42A34247DC1A15D14C3E
:10BA80001B031B0B9846A4468024CF4B64034344FE
:10BA90002340CE4C624452195C4045461B159946E2
:10BAA0002543CA4B290091440022FFF749F9434638
:10BAB00002331B0306000F001B0B0022022B2FDC9E
:10BAC0000023FDF731FD002800D1C1E04B46002BDB
:10BAD00000D14CE14846FFF79DFCBD4ABD4B040038
:10BAE0000D00FEF7ADFEBC4A06000F00BB4B200068
:10BAF0002900FEF7A5FE02000B0030003900FDF71B
:10BB00005BFF07E0AE4C0025A342B7DD02000B004F
:10BB1000FDF752FF08B01CBC90469946A246F0BD06
:10BB20008023DB05FDF748FF02000B0030003900E1
:10BB3000FEF752FA040048460D00FFF76BFC2200A6
:10BB4000029003912B002000290004940595FEF734
:10BB500077FE04000D00A24B020043449A460B00FE
:10BB600000940195FEF76CFE04000D009D4A9E4B6B
:10BB7000FEF766FE9D4A9E4BFDF71EFF22002B003E
:10BB8000FEF75EFE9B4A9C4BFDF716FF22002B0042
:10BB9000FEF756FE994A9A4BFDF70EFF009A019B5D
:10BBA000FEF74EFE974A00900191974B2000290026
:10BBB000FEF746FE954A964BFDF7FEFE22002B004F
:10BBC000FEF73EFE934A944BFDF7F6FE22002B0053
:10BBD000FEF736FE0B00020000980199FDF7ECFE1F
:10BBE0000D0041468D4B04005B1A51460B43002B60
:10BBF00054DD00228A4B30003900FEF721FE32006E
:10BC00003B00FEF71DFE4B460A0001000091019229
:10BC1000002B72D11300290002002000FDF7CCFE9A
:10BC2000049A059BFEF70CFE02000B000098019998
:10BC3000FFF786F802000B0030003900FFF780F8AC
:10BC400068E70022002300207649FEF7C5F961E786
:10BC5000754A764B30003900FEF7F2FD02000B000A
:10BC600000206F49FFF76CF8320004000D003B0024
:10BC700030003900FEF7E4FD0B000200290020002F
:10BC8000FEF7DEFD4B4604000D00002B72D10200D2
:10BC90000B0030003900FFF753F83BE74B46002B11
:10BCA00000D1C5E002980399494A4A4BFEF7C8FD06
:10BCB0002200009001912B0030003900FFF740F87E
:10BCC000049A059BFEF7BCFD434A04000D00029850
:10BCD0000399424BFEF7B4FD02000B00200029003F
:10BCE000FFF72EF832003B00FFF72AF802000B00A6
:10BCF00000980199FFF724F80CE7354A354B029874
:10BD00000399FEF79DFD009A019B06900791200084
:10BD10002900FDF751FE049A059BFEF791FD2E4A7E
:10BD200004000D00029803992C4BFEF789FD0200D8
:10BD30000B0020002900FDF73FFE02000B000098D9
:10BD40000199FEF7FDFF32003B00FEF7F9FF02000C
:10BD50000B0006980799FEF7F3FFDBE602000B00E5
:10BD6000FEF7EEFF00220023FEF736F9D2E60020B0
:10BD70000021CFE64846FFF74DFB154A154B0090D2
:10BD80000191FEF75DFD144A02900391009801991C
:10BD9000124BFEF755FD02000B0020002900FEF7B4
:10BDA000CFFF32003B00FEF7CBFF02000B000298F2
:10BDB0000399FEF7C5FFADE6FFFF0F0000005043FB
:10BDC000FFFFEF7F01FCFFFF645F09000000F03F11
:10BDD0000000E0FE422EE63F763C7935EF39EA3D41
:10BDE00086EBF9FF44523EDF12F1C23FDE03CB96F1
:10BDF0006446C73F599322942449D23F93555555E1
:10BE00005555E53F9FC678D0099AC33FAF788E1D40
:10BE1000C571CC3F04FA97999999D93F51B806005A
:10BE20000000E03F000050C3555555555555D53FCE
:10BE300022002B0030003900FEF782FF049A059B98
:10BE4000FEF7FEFCF6E6C0460020704700200149E0
:10BE50007047C0460000F87F014B18687047C04625
:10BE600028F0FF1F8025000040380000004B000034
:10BE7000807000000096000000E10000002C01002E
:10BE800000C201000084030090D0030020A107003D
:10BE900040420F0000000000E0930400C0270900AA
:10BEA000FF0000010000000032FF0000E803000076
:10BEB0001027000088130000D00700000A000000CF
:10BEC0000000000000C2EB0B000001006400000055
:10BED0006400000000070000F40100000000000002
:10BEE0000050C30000881300014008080000000053
:10BEF00000000000C80000000100000000800000F9
:10BF0000C800000000000000000000000000000069
:10BF10000000000000000000000000000000000021
:10BF2000000000000101010001000000000000000D
:10BF30000000000000000100000000000000000000
:10BF400000000000010101000000000000000000EE
:10BF500000010000000000000101010001010001DA
:10BF600001000000000000000000000000000000D0
:10BF700000000000000000000000000000000000C1
:10BF800000000000000000000000000000000101AF
:10BF9000000000010001000100000000000000009E
:10BFA00000000000D0A10000B2A100006CA10000C0
:10BFB0008AA000006CA10000A4A100006CA10000F8
:10BFC0008AA00000B2A10000B2A10000A4A100005C
:10BFD0008AA0000082A0000082A0000082A00000D1
:10BFE000E8A3000030AA0000F0A80000F0A80000BC
:10BFF000ECA8000008AA000008AA0000FAA90000A6
:10C00000ECA8000008AA0000FAA9000008AA000095
:10C01000ECA8000010AA000010AA000010AA00005E
:10C0200014AC00003132333156313136000000009B
:10C030006C6F670000000000F8B5C046F8BC08BC93
:10C040009E467047F8B5C046F8BC08BC9E4670478F
:04C05000392400008F
:04C0540011240000B3
:10C0580024C00000010200000000000000000000F1
:10C0680000000000080002000100000000000000BD
:10C07800000000000024F4002CF0FF1F0000000066
:10C0880000000000000000000000000000000000A8
:10C098000000000000000000000000000000000098
:10C0A8000000000000000000000000000000000088
:10C0B8000000000000000000000000000000000078
:10C0C8000000000000000000000000000000000068
:10C0D8000000000000000000000000000100000057
:04C0E8000000000054
:040000030000B851F0
:00000001FF
